:020000040800F2
:1000000000060020B5050008791A00082D1A00081E
:10001000551A00082D1A00084D1A0008B7050008E7
:10002000B7050008B7050008B7050008154C00081B
:10003000B7050008B7050008B7050008B7050008B0
:10004000B7050008B7050008B7050008B7050008A0
:10005000B7050008B705000899620008C5620008E6
:10006000F16200081D63000849630008B705000835
:10007000B7050008B7050008B7050008B705000870
:10008000B7050008B7050008B7050008B705000860
:10009000B7050008B7050008B70500087563000834
:1000A000B7050008B7050008B7050008B705000840
:1000B000B7050008B7050008B7050008B705000830
:1000C000B7050008B7050008B7050008B705000820
:1000D000B705000861640008B7050008B705000807
:1000E000D9630008B7050008B7050008B705000880
:1000F000B7050008B7050008B7050008B7050008F0
:10010000B7050008B705000889640008B7050008AE
:10011000B7050008B7050008B7050008B7050008CF
:10012000B7050008B7050008B7050008B7050008BF
:10013000B7050008B7050008B7050008B7050008AF
:10014000B7050008B7050008B7050008B70500089F
:10015000B7050008B7050008B7050008B70500088F
:10016000B7050008B7050008B7050008B70500087F
:10017000B705000835590008B7050008B70500089D
:10018000B7050008B705000875640008B705000842
:10019000B7050008B7050008B7050008B70500084F
:1001A000B7050008B7050008B7050008B70500083F
:1001B0004D640008B7050008B7050008B70500083A
:1001C000B7050008B7050008B7050008B70500081F
:1001D000B705000821590008B7050008B705000851
:1001E000B7050008B7050008B7050008B7050008FF
:1001F000B7050008B7050008B7050008B7050008EF
:10020000B7050008B7050008B7050008B7050008DE
:10021000B7050008B7050008B7050008B7050008CE
:10022000B7050008B7050008A54D0008B705000888
:10023000B7050008B7050008B7050008B7050008AE
:10024000B7050008B7050008B7050008B70500089E
:10025000B7050008B7050008B7050008B70500088E
:10026000B7050008B7050008B7050008B70500087E
:10027000B7050008B7050008B7050008B70500086E
:10028000B7050008B7050008B7050008B70500085E
:10029000B7050008B7050008B7050008B70500084E
:1002A0009D070008011A0008E5240008000000006E
:1002B00053B94AB9002908BF00281CBF4FF0FF31CD
:1002C0004FF0FF3000F074B9ADF1080C6DE904CEC9
:1002D00000F006F8DDF804E0DDE9022304B0704721
:1002E0002DE9F047089D04468E46002B4DD18A42E9
:1002F000944669D9B2FA82F252B101FA02F3C2F11C
:10030000200120FA01F10CFA02FC41EA030E9440AC
:100310004FEA1C48210CBEFBF8F61FFA8CF708FBCD
:1003200016E341EA034306FB07F199420AD91CEBA5
:10033000030306F1FF3080F01F81994240F21C81D7
:10034000023E63445B1AA4B2B3FBF8F008FB10331F
:1003500044EA034400FB07F7A7420AD91CEB040454
:1003600000F1FF3380F00A81A74240F20781644424
:10037000023840EA0640E41B00261DB1D4400023A9
:10038000C5E900433146BDE8F0878B4209D9002D0D
:1003900000F0EF800026C5E9000130463146BDE897
:1003A000F087B3FA83F6002E4AD18B4202D3824201
:1003B00000F2F980841A61EB030301209E46002DB0
:1003C000E0D0C5E9004EDDE702B9FFDEB2FA82F205
:1003D000002A40F09280A1EB0C014FEA1C471FFA63
:1003E0008CFE0126200CB1FBF7F307FB131140EA4A
:1003F00001410EFB03F0884208D91CEB010103F117
:10040000FF3802D2884200F2CB804346091AA4B2D8
:10041000B1FBF7F007FB101144EA01440EFB00FEAC
:10042000A64508D91CEB040400F1FF3102D2A64511
:1004300000F2BB800846A4EB0E0440EA03409CE7B0
:10044000C6F12007B34022FA07FC4CEA030C20FA5D
:1004500007F401FA06F31C43F9404FEA1C4900FA7D
:1004600006F3B1FBF9F8200C1FFA8CFE09FB1811FA
:1004700040EA014108FB0EF0884202FA06F20BD96D
:100480001CEB010108F1FF3A80F08880884240F2BD
:100490008580A8F102086144091AA4B2B1FBF9F001
:1004A00009FB101144EA014100FB0EFE8E4508D9FC
:1004B0001CEB010100F1FF346CD28E456AD9023881
:1004C000614440EA0840A0FB0294A1EB0E01A14266
:1004D000C846A64656D353D05DB1B3EB080261EBD4
:1004E0000E0101FA07F722FA06F3F1401F43C5E9AE
:1004F000007100263146BDE8F087C2F12003D840E4
:100500000CFA02FC21FA03F3914001434FEA1C4725
:100510001FFA8CFEB3FBF7F007FB10360B0C43EA17
:10052000064300FB0EF69E4204FA02F408D91CEBC7
:10053000030300F1FF382FD29E422DD902386344C5
:100540009B1B89B2B3FBF7F607FB163341EA034165
:1005500006FB0EF38B4208D91CEB010106F1FF38B4
:1005600016D28B4214D9023E6144C91A46EA0046AB
:1005700038E72E46284605E70646E3E61846F8E63D
:100580004B45A9D2B9EB020864EB0C0E0138A3E786
:100590004646EAE7204694E74046D1E7D0467BE767
:1005A000023B614432E7304609E76444023842E7DF
:1005B000704700BF02E000F000F8FEE772B63A486C
:1005C00080F30888394880F3098839484EF6085185
:1005D000CEF20001086040F20000CCF200004EF6BE
:1005E0003471CEF200010860BFF34F8FBFF36F8FFD
:1005F00040F20000C0F2F0004EF68851CEF2000149
:100600000860BFF34F8FBFF36F8F4FF00000E1EE34
:10061000100A4EF63C71CEF200010860062080F30D
:100620001488BFF36F8F04F0B3FB04F055FB05F0A3
:10063000F1FB4FF055301F491B4A91423CBF41F836
:10064000040BFAE71C49194A91423CBF41F8040BDC
:10065000FAE71A491A4A1B4B9A423EBF51F8040B5B
:1006600042F8040BF8E700201749184A91423CBFB2
:1006700041F8040BFAE704F06DFB05F041FC144C63
:10068000144DAC4203DA54F8041B8847F9E700F034
:100690004FF8114C114DAC4203DA54F8041B884753
:1006A000F9E704F055BB00000006002000220020FE
:1006B000000000080000002000060020D06C0008A8
:1006C00000220020CC220020D0220020684E0020F2
:1006D000A0020008AC020008AC020008AC0200084E
:1006E0002DE9F04F2DED108AC1F80CD0D0F80CD0C8
:1006F000BDEC108ABDE8F08F002383F311882846F3
:10070000A047002003F0BCFCFEE703F0EBFB00DF9A
:10071000FEE70000054B10B504460360806810B189
:1007200003685B689847204610BD00BF90680008CA
:1007300038B504F095F9054604F062FA0446F0B9BC
:10074000144B9D421DD001339D4241F2883512BFAA
:10075000044600250124002004F08CF90CB100F0BF
:100760009FF80D4C00F042FF00F0C2FD204601F062
:10077000F1FC40B944F6206003F088FCF6E7002560
:10078000E9E70546E7E7284600F046F900F088F873
:10079000F9E700BF010007B0D02200200448054B54
:1007A000054A036000230549836005F0CBBE00BF06
:1007B000D022002090680008FC24002015070008C3
:1007C00008B500F061FDA0F120035842584108BD72
:1007D00007B5042101900DEB010000F073FD03B09B
:1007E0005DF804FB07B541F21203022101A8ADF840
:1007F000043000F067FD03B05DF804FB38B520233A
:1008000083F311881748C3680BB103F0D7FC0023AA
:10081000154A4FF47A71134803F094FC002383F3D4
:100820001188124C236813B12368013B236063686D
:1008300013B16368013B63600D4D2B7833B9636876
:100840007BB9022000F012FE322363602B78032B69
:1008500007D163682BB9022000F008FE4FF47A73C9
:10086000636038BD60230020FD0700087C24002061
:1008700074230020084B187003280CD8DFE800F020
:1008800008050208022000F0E9BD022000F0DCBDEE
:10089000024B00225A607047742300207C24002001
:1008A000F7B5564801A901F0CDFD002800F0A3805E
:1008B000534B544A1C461968013100F099800433A7
:1008C0009342F8D16268504B9A4240F291804F4B6C
:1008D000DB6803F1104303F580139A4280F08880AF
:1008E000002000F01FFD0220FFF7C4FF484B00214D
:1008F000D3F8E820C3F8E810D3F81021C3F810119A
:10090000D3F81021D3F8EC20C3F8EC10D3F814215D
:10091000C3F81411D3F81421D3F8F020C3F8F01061
:10092000D3F81821C3F81811D3F81821D3F8802070
:1009300042F00062C3F88020D3F8802022F00062E9
:10094000C3F88020D3F88020D3F8802042F00072D2
:10095000C3F88020D3F8802022F00072C3F88020F2
:10096000D3F8803072B64FF0E023C3F8084DD4E9D5
:100970000004BFF34F8FBFF36F8F264AC2F8841075
:10098000BFF34F8F536923F480335361BFF34F8F0D
:10099000D2F8803043F6E076C3F3C905C3F34E3393
:1009A0005B0103EA060C29464CEA81770139C2F85B
:1009B0007472F9D2203B13F1200FF2D1BFF34F8FA5
:1009C000BFF36F8FBFF34F8FBFF36F8F536923F464
:1009D000003353610023C2F85032BFF34F8FBFF38F
:1009E0006F8F202383F31188854680F30888204782
:1009F000024801F087F803B0F0BD00BFD02200200C
:100A00000000109020001090FFFF0F9000220020A7
:100A10000044025800ED00E02DE9F04FB34B9FB0C9
:100A20002022FF21089016A89E68DB68079300F03B
:100A300087FDAF4A1378A3B90121AE481170C36096
:100A4000202383F31188C3680BB103F0B7FB0023A5
:100A5000A94A4FF47A71A74803F074FB002383F38B
:100A60001188089B13B1A54B089A1A60A44A137801
:100A7000032B03D000231370A04A53600023089D6A
:100A8000A04F98469B46CDE90533012000F0E6FCD7
:100A900025B19A4B1B68002B00F08783002000F0E3
:100AA000F3FB0E900E9B002BF2DB012000F0CCFC40
:100AB0000E9B213B1F2BE8D801A252F823F000BF68
:100AC000410B0008690B0008030C00088B0A0008A2
:100AD0008B0A00088B0A0008EF0E0008ED100008D2
:100AE000850F00086B10000891100008B71000086F
:100AF0008B0A0008C91000088B0A0008351100088D
:100B0000E10B00088B0A0008B1110008A10C0008D5
:100B1000D90D00088B0A0008E10F00088B0A0008B5
:100B20008B0A00088B0A00088B0A00088B0A000851
:100B30008B0A00088B0A00088B0A0008030C0008C7
:100B40000220FFF73DFE002840F05B83089B022156
:100B5000069A11A8002A08BF1D4641F21233ADF8CB
:100B6000443000F0AFFB90E74FF47A7000F08CFB5C
:100B7000041EEBDB0220FFF723FE0028E6D0013C39
:100B8000052C00F24083DFE804F0030A0D1013394E
:100B90000523042111A8119300F094FB17E0042110
:100BA0005248F9E704215848F6E704215748F3E78B
:100BB0004FF01C09484609F1040900F0B5FB042177
:100BC000119011A800F07EFBB9F12C0FF2D1012099
:100BD000059B4FF0000B00FA04F41C43E3B20593AD
:100BE00000F0FAFCB8F1000F05D0059B03F00B03F1
:100BF0000B2B08BF0025FFF7F5FD46E7042144480D
:100C0000CAE7B8F1000FA1D0059B03F00B030B2B33
:100C10009CD10220FFF7D4FD0446002896D0012085
:100C20004FF0000800F07EFB0220FFF723FE5FFA82
:100C300088F9484600F086FB0546B8B10E9948464B
:100C400008F10108A1F140025142514100F08AFB34
:100C50000028ECD10546069441F21213022111A896
:100C6000A046ADF8443000F02DFB0EE72E46DFF82D
:100C70007C800120FFF7FEFDD8F80830B34207D989
:100C8000304600F051FB013040F0C0820436F3E7FB
:100C900000261B4BA04606941E70184B5E609FE713
:100CA000B8F1000F3FF452AF059B03F00B030B2B81
:100CB0007FF44CAF64210FA800F0FAFA81460028B7
:100CC0007FF444AF0220FFF77BFD044600283FF489
:100CD0003DAF3A6A7B6A0F9953438DF837908B4248
:100CE0001AD20C4800F0CCFB30E700BF00220020F5
:100CF0007824002060230020FD0700087C240020C9
:100D000074230020D022002004220020082200208A
:100D10000C220020886600084FF4801AAC48C846B0
:100D2000BAFBF2FA00F0ACFBFFF75CFD01210DF11C
:100D3000370000F0C7FA0F9B434541D9002310AAA2
:100D400051463846CDE9103311AB00F0DFFE0028E4
:100D500082D000F099FE109B00EB030901210DF1F8
:100D6000370000F0AFFA00F08FFE484520D9384632
:100D700001F002F980B964210F9B96480AF1010A3B
:100D800001FB08F1B1FBF3F18DF83710C9B200F0A7
:100D900077FB3B6A9844CEE700F076FE119B18443F
:100DA00048453FF659AF00F06FFE109B00EB03097A
:100DB000109B4FF47A70A3FB000303F067F9CDE7B3
:100DC000642301210DF13700A0468DF8373000F083
:100DD00079FA0023079303E7B8F1000F3FF4B6AEAA
:100DE000059B03F00B030B2B7FF4B0AE0220FFF743
:100DF00041FD322000F048FAB0F1000AFFF6A6AE3D
:100E0000079BD14653440993734B099ADB689A4276
:100E10003FF69CAEBAF5807F3FF798AE6F4A00244C
:100E2000A2450A920EDD4FF47A7000F02DFA0E9072
:100E30000E9B002BFFF68AAE0E9B01340A9A02F835
:100E4000013BEDE7C820FFF7BBFC044600283FF458
:100E50007DAE079B1F2B11D8C3F1200223F00300A6
:100E600016AB5E495245184428BF52460A9200F01C
:100E700035FB0A9AFF21594800F062FB002398468F
:100E8000CDE91033079B03F580130B93B9F1000FE5
:100E900002D1A046099B9DE711AB504A0B993846F9
:100EA000029310AB4244414401930FAB00934B4675
:100EB00001F034FA00283FF4CFAE00F0E7FD0F9BBD
:100EC00082460A919844A9EB030900F0DFFD109BCC
:100ED0000A9A13EB0A0342F10002834272EB010308
:100EE000F3D2384601F048F80028EED1CEE7B8F149
:100EF000000F3FF42BAE059B03F00B030B2B7FF48D
:100F000025AE0220FFF7B6FC322000F0BDF9B0F1AB
:100F1000000AFFF61BAE1AF003047FF417AE2E4A48
:100F20000AEB0603926893423FF610AEBAF5807F53
:100F30003FF70CAEDFF8A490A2450DDD4FF47A70B8
:100F400000F0A2F90E900E9B002BFFF6FFAD0E9B5A
:100F5000013409F8013BEFE7C820FFF731FC0446F4
:100F600000283FF4F3ADCAF387021C4930464FEA2C
:100F7000AA0900F0EDFA804600283FF46DAE06EBBA
:100F800089062DE60220FFF71BFC00283FF4DEADAA
:100F900000F006FA00283FF4D9AD4FF00009DFF861
:100FA00038A04C46DAF808304B450CD9484609F1D0
:100FB000040900F0B9F90422119011A9204601F0AA
:100FC000B7FA0446EEE72046FFF702FC08E600BF4A
:100FD000AD660008C56600080022002078230020C6
:100FE000642110A800F064F9044600287FF4AEAD37
:100FF0000220FFF7E5FB00283FF4A8AD109BA146B7
:1010000003F0030A1099A1EB0A01A1421BD91F2C7E
:1010100011D8169B01330ED024F003031EAA1344EB
:1010200053F8203C11934846042211A9043401F0DE
:101030007FFA8146E6E7042311AA04F580113846B9
:1010400001F0B8F9EFE7BAF1000F0CD0534611AA3E
:1010500001F58011384601F0ADF94846524611A914
:1010600001F066FA81464846AEE70023642111A8E4
:10107000119300F01DF900287FF468AD0220FFF7FE
:101080009FFB00283FF462AD119800F07FF99BE7C9
:101090000023642111A8119300F00AF900287FF4BD
:1010A00055AD0220FFF78CFB00283FF44FAD11989F
:1010B00000F06EF988E70220FFF782FB00283FF47A
:1010C00045AD00F07DF97FE70220FFF779FB0028AE
:1010D0003FF43CAD11A9142000F078F90990FFF716
:1010E00077FB099911A800F0EDF879E5322000F0BE
:1010F000CBF8041EFFF62AADA3077FF427AD444AC0
:1011000004EB0B03926893423FF620AD0220FFF7F9
:1011100057FB00283FF41AAD24F003045C44A345B8
:101120003FF45EAD58460BF1040B00F0FDF8FFF7FD
:101130004FFBF4E74FF47A70FFF742FB00283FF4CF
:1011400005AD00F02DF980B1169B013328D011AB0D
:1011500016AA4FF480113846029310AB01930FABDF
:101160000093202301F0DAF808B9444674E500F052
:101170008DFC284E04460D4600F088FC109B1B1980
:1011800045F10002834272EB0103F5D2304600F0D4
:10119000F3FE0028F0D12022FF2116A800F0D0F99C
:1011A000FFF720FB1C4802F071FF1FB0BDE8F08F75
:1011B000B8F1000F3FF4CAAC059B03F00B030B2BF7
:1011C0007FF4C4AC0023642111A8119300F070F8DF
:1011D000044600287FF4BAAC0220FFF7F1FA8146FA
:1011E00000283FF4B3ACFFF7FDFA41F2883002F07B
:1011F0004DFF119800F038FAC846254600F0ECF98A
:1012000043E48046ECE44FF0000B9FE4069423E5B2
:1012100000220020D0220020A08601002DE9F84FF6
:101220004FF47A7306460D46002402FB03F7DFF8FD
:101230005080DFF8509098F900305FFA84FA5A1C19
:1012400001D0A34210D159F824002A463146036840
:10125000D3F820B03B46D847854205D1074B012043
:1012600083F800A0BDE8F88F0134032CE3D14FF4DC
:10127000FA7002F00BFF0020F4E700BFC824002042
:101280001022002014220020002307B5024601216D
:101290000DF107008DF80730FFF7C0FF20B19DF872
:1012A000070003B05DF804FB4FF0FF30F9E70000E2
:1012B0000A46042108B5FFF7B1FF80F00100C0B273
:1012C000404208BD074B0A4630B41978064B53F824
:1012D0002140014623682046DD69044BAC4630BC02
:1012E000604700BFC824002014220020A08601000F
:1012F00070B50A4E00240A4D03F098F93080286832
:101300003388834208D903F08DF92B6804440133F4
:10131000B4F5003F2B60F2D370BD00BFCA2400209B
:101320008424002003F036BA00F1006000F500309C
:101330000068704700F10060920000F5003003F093
:10134000ADB90000054B1A68054B1B889B1A8342F8
:1013500002D9104403F066B90020704784240020AD
:10136000CA24002038B50446074D29B12868204416
:10137000BDE8384003F062B92868204403F058F90A
:101380000028F3D038BD00BF84240020002070471F
:1013900000F1FF5000F58F10D0F8000870470000F2
:1013A000064991F8243033B100230822086A81F8F5
:1013B0002430FFF7BFBF0120704700BF8824002002
:1013C000014B1868704700BF0010005C1B4B0246C1
:1013D000F0B518681A4BC0F30B06000C1F885C6848
:1013E000BE4293F9085003D09F89BE4203D10C330B
:1013F0005C6893F908500426124B1F880433874217
:1014000008BF13F9025C013EF7D1013A013C0B46DB
:101410000A44934207D214F9016F581C2EB10346B7
:1014200000F8016CF5E7184605E02C2482421C7098
:1014300001D9981C5D70401AF0BD00BF0010005C1F
:1014400020220020F0660008022803D1024B4FF44E
:1014500000329A61704700BF00000258022801D193
:10146000014B9861704700BF00000258022804D168
:10147000024A536983F00203536170470000025827
:101480000FB4124B30B51A78B5B042B901221049E9
:1014900010481A704FF461430B6001F0B1FE39AB94
:1014A0000C4C389AC82102A8019300F0BDFA2368B9
:1014B000C8280246DD6902A9074B28BFC82220467A
:1014C000A84735B0BDE8304004B07047CC240020B8
:1014D000D024002094250020A0860100002310B510
:1014E000934203D0CC5CC4540133F9E710BD000033
:1014F000013810B510F9013F3BB191F900409C4211
:1015000003D11AB10131013AF4E71AB191F900207F
:10151000981A10BD1046FCE70138013910F9013F57
:1015200011F9012F0BB19342F8D0981A70470000BF
:1015300003460246D01A12F9011B0029FAD170475E
:1015400002440346934202D003F8011BFAE77047B6
:101550002DE9F8431F4D14460746884695F8242088
:1015600052BBDFF870909CB395F824302BB9202241
:10157000FF2148462F62FFF7E3FF95F8240041461C
:10158000C0F1080205EB8000A24228BF2246D6B275
:101590009200FFF7A3FF95F82430A41B17441E44C4
:1015A0009044E4B2F6B2082E85F82460DBD1FFF750
:1015B000F7FE0028D7D108E02B6A03EB82038342B1
:1015C000CFD0FFF7EDFE0028CBD10020BDE8F88397
:1015D0000120FBE788240020024B1A78024B1A7086
:1015E000704700BFC824002010220020F8B5184C16
:1015F000184801F0A7FE2146164801F0CFFE2468E6
:101600001548D4F89020154ED2F80438144D43F004
:101610000203104FC2F8043802F038FD2046114989
:1016200001F0CAFFD4F890200324D2F8043823F044
:101630000203C2F804384FF4E133336055F8040B69
:10164000B84202D0314601F0DBFD013CF6D1F8BDD5
:10165000206A0008D02F002040420F00B024002054
:1016600014220020286A00080C4B70B50C4D04466B
:101670001E780C4B55F826209A420DD00A4B0021BB
:1016800018221846FFF75CFF0460014655F8260053
:10169000BDE8704001F0B4BD70BD00BFC82400209B
:1016A00014220020D02F0020B024002038B5084B91
:1016B00004461546017543600A21243003F00EFAF2
:1016C00004F128002A460A2103F008FA204638BD12
:1016D000D8680008F8B51E461B6805460C46174634
:1016E0001BB9236863B9012408E0BDF8182031460E
:1016F000806A03F00BFA0028F3D100242046F8BDDD
:1017000021463A46686A03F037FA04460028EAD1CF
:101710003368002BF1D0A86A03F062FAEEE700000C
:1017200038B50D46114604461A4611B1806A03F0D9
:1017300015FA2DB12946606ABDE8384003F048BA71
:1017400038BD00007047000070470000002070475F
:101750000020704713B56C4600F1140384E80600BE
:1017600094E8030083E8050002B010BD0020704734
:1017700013B56C4600F10C0384E8060094E80300FE
:1017800083E8050002B010BD0023C0E903337047B1
:1017900082B002AB03E9060002B070477047000058
:1017A00000207047704700000020704700207047FD
:1017B0000120704782B0002002A901E90C0002B0AC
:1017C0007047000000207047002070470B6883635B
:1017D0004B6843638B68C363CB6803640B694364E2
:1017E0007047000038B5036B0446154D1B7955F85A
:1017F000330002F0DDF9D4E90B231B7955F83310DF
:1018000002F130034968994218D000231363E26A59
:101810005363D4E90B12537C581E137C92681B044B
:1018200043EA002313438B63D4E90B131B79303154
:1018300055F83300BDE8384002F04EB938BD00BF5E
:101840005C670008F8B51D4F05460E46114638681E
:10185000FFF762FE78BB74683B7924B394F82C20C0
:101860009A420BD02468F8E70122B521FFF71EFF4A
:10187000736823603B79746084F82C30482004F04E
:101880006BFE68B100220271C0E90322C0E90522A3
:10189000027A42F007020272094AC0E90B4702606D
:1018A00028602846F8BD402004F056FE0446002873
:1018B000DAD12C60F5E700232B60F2E7E824002062
:1018C0006C670008044B10B504460360406A08B119
:1018D00004F040FE204610BD1067000810B5044615
:1018E000FFF7F0FF204604F033FE204610BD000055
:1018F00008B519B1FFF776FF012008BD036B1A790F
:10190000024B53F8320002F057F9F5E75C67000824
:101910002DE9FF41DDF828800546174603911FFA9F
:1019200088F60293FFF75EFF02ABBAB203A9E86A3A
:101930000096FFF7CFFE044638B900212846FFF78E
:10194000D7FF204604B0BDE8F081AFB92B6B05F19D
:1019500034011A79134B53F83200B8F1000F19D142
:1019600002F0C8F880F00104E4B23346E86ADDE929
:101970000221FFF7D5FEE0E7029B83B92B6B3A46C5
:10198000084805F134011C79039B50F8340002F03B
:10199000C7F8E7E7029B424602F0D8F8E2E70024E6
:1019A000E3E700BF5C67000813B504460191FFF749
:1019B00019FF019A236B04F134011879054B53F890
:1019C000300002F0D9F800212046FFF791FF0120F6
:1019D00002B010BD5C67000810B50446FFF702FFB7
:1019E000236B1A79054B53F8320002F0D3F800212B
:1019F0002046FFF77DFF012010BD00BF5C67000897
:101A0000064B0121064A1A6000221A71054AC3E9F1
:101A1000021240F217221A82704700BFE824002009
:101A200000670008000E270700F07ABF00B59BB0E2
:101A3000EFF3098168226846FFF750FDEFF3058355
:101A4000014B9B6BFEE700BF00ED00E008B5FFF720
:101A5000EDFF000000B59BB0EFF3098168226846F6
:101A6000FFF73CFDEFF30583014B5B6BFEE700BF27
:101A700000ED00E0FEE70000FEE700000FB408B54F
:101A8000029802F093FAFEE702F08ABF02F062BF0A
:101A900080697047C0697047006A7047406A704744
:101AA000806A7047F0B5ADF2044D0E460546002140
:101AB0004FF47F7201A80091FFF742FD2C6A744336
:101AC00001362B6A7343A34216D92B686A46214616
:101AD00028465F684FF48063B84770B16A464FF498
:101AE000806312F8011BFF290AD1013B9BB2002B36
:101AF000F7D104F58064E4E701200DF2044DF0BD58
:101B00000020FAE780680368DB69184730B5456A4A
:101B100085B004468D420FD30568CDE90023026AE3
:101B200003ABAD6A5143A84720B1206A039BC31A97
:101B30005842584105B030BD0020FBE7F0B5C569FB
:101B400087B004468D4212D30C9F866905687143A5
:101B5000CDE9013705AB00936D69036AA84720B151
:101B6000A069059BC31A5842584107B0F0BD002038
:101B7000FBE70000F0B5662389B0002405464FF46A
:101B800080768068079403A9CDE90336CDE9054442
:101B900003685B699847A868224621460368009459
:101BA0001F692346B847A8689923079403A9CDE97C
:101BB0000336CDE9054403685B699847A868224667
:101BC0002146036800941D692346A84709B0F0BD6B
:101BD000254B2DE9F04F1B789FB0002504468DF86A
:101BE00028304FF09F0E80684FF00123ADF8295048
:101BF00005A90995CDE905E3CDE9075503685B69BA
:101C00009847A06803222946036800922A461E6965
:101C10000AABB04728B394F88C20144B9DF82810D9
:101C200003EBC2031A7991421BD19DF829205B79FD
:101C30009A4216D1A0684FF05A0C0D4B082605A900
:101C40000996CDE905C3CDE9075503685B69984757
:101C5000A0682A462946036800961F690AABB84760
:101C600040B9002048E100BF7066000870680008B5
:101C7000002500010422B1490AA804F09DFC054694
:101C80000028EED1BDF82C306FF48277A3813B445D
:101C9000012BE6D8079605A9CDE90A00A0680368DC
:101CA0005B699847A0682A462946036800961E6922
:101CB0000AABB0470028D4D0DDE90A361A0202F494
:101CC000706242EA1662FF2ACBD11B0E26F07F46D5
:101CD00050222946142B26610AA828BF1423A37377
:101CE000FFF72EFCA068079605A903685B69984773
:101CF000A068A37B294602689B0000930AAB166983
:101D00002A46B0470028ACD00B990029A9DBC908A6
:101D10006FF07E43149D4FF0010E994228BF194683
:101D2000C5F303130EFA03F221FA03F30391616181
:101D3000A261E361002B94D02646A44600274FF011
:101D400002081EAAC7F3460302EB830353F834AC20
:101D500007F001031B01DA1D0EFA03F908FA02F27B
:101D6000A2EB090202EA0A02DA401AD003F10809DA
:101D70000F330EFA02F2216A08FA03F30EFA09FB96
:101D8000CCF830208A42A3EB0B0B0BEA0A0A2AFAA2
:101D900009F98CF82C90A36A88BF2262934288BF0D
:101DA000A26201370CF1100C042FCAD1236A4FF044
:101DB000020C039A4FF0010E139F9A4224BFB2FB0C
:101DC000F3F1616207F00F0138BF01234FF0090200
:101DD00001F1010138BF63624900336B33B3531C17
:101DE0000EFA02F8A2F105090CFA03F30EFA09FA49
:101DF000A3EB080302F1FF380CFA08F83B40A8EB0C
:101E00000A08D34008EA070828FA09F877D0012B16
:101E100077D0022B77D0032B08BF4FF47A735FFA89
:101E200088F808FB033373634B43B3630732103600
:101E3000252AD2D115F0C04FC5F3417365D0012BCF
:101E400065D0022B0CBF4FF47A634FF47A43C5F38D
:101E5000046202FB0333E3664B432367199B9E072F
:101E600058D0062384F8743015F4005F05F00F0392
:101E7000C5F3042514BF40220822013305FB0225C7
:101E80005B00A5675D430A9B9F02E5677FF5E9AEAE
:101E90000C9B1A0A84F88020C3F3421203F01F033C
:101EA00084F8882084F88130189BC3F3025213F41D
:101EB000401F84F883207FF4D4AEDE0602D5042AC6
:101EC0007FF4CFAE03F40072002A14BF0122002277
:101ED00084F8872004D0DD0324D5002384F88930DA
:101EE000179B1A0722D5002384F88630702384F8C4
:101EF0008530012384F88D301FB0BDE8F08F0123B9
:101F00008DE710238BE7802389E710239FE74FF4A9
:101F100080739CE7590701D55023A3E713F0780F8E
:101F2000A2D09EE69903DBD50123D7E75B07E0D576
:101F3000012384F886300523D9E700BFCC67000869
:101F400030B58BB000240546806803924FF0012223
:101F5000059105A9CDE90624CDE908440268526936
:101F60009047A8680121039B0268009121461569EA
:101F70002246A8470BB030BD13B504460DF1070249
:101F800090F88510FFF7DCFF94F886309DF8070085
:101F90001BB100F0010002B010BDC043C0F3C0107F
:101FA000F9E7000030B54FF001238BB0002405465F
:101FB00080688DF80F20059105A9CDE90634CDE99B
:101FC000084403685B699847A86801220DF10F0176
:101FD000036800941D692346A8470BB030BD00007C
:101FE000F7B517460DF1070206461D46FFF7A8FF95
:101FF00068B19DF8074039469DF82020304624EA14
:1020000005042A4022438DF80720FFF7CBFF03B0D9
:10201000F0BD000030B54FF4807389B00024054650
:102020008068039103A9CDE90434CDE9064403682F
:102030005B699847A86822462146036800941D6999
:102040002346A84709B030BD10B504462368204692
:10205000DB6A98470028F9D110BD000010B590F850
:10206000743004465BB1FFF7EFFF012394F874105E
:10207000204684F88E30BDE81040FFF7CBBF01202A
:1020800010BD000010B590F87430044653B1FFF74E
:10209000DBFF01232046042184F88E30BDE8104088
:1020A000FFF7B8BF012010BD70B590F883308AB03B
:1020B0000446042B48D10DF10E020521FFF740FF25
:1020C00000282FD00DF10F0235212046FFF738FFF1
:1020D00040B320461E4EFFF7C1FF2046FFF7B4FF76
:1020E00005AD0FCE0FC5336805A99DF80E202B60F6
:1020F0009DF80F30A06843F002038DF810208DF892
:102100000F308DF8113003685B699847A068002391
:1021100004A90268009315690222A84728B920463D
:10212000FFF7B0FF00200AB070BD2046FFF7AAFFFE
:102130000DF10F0235212046FFF702FF0028F1D0F4
:102140009DF80F309B07EDD501202071EBE700BF14
:10215000746600082DE9F341002304468068A360FB
:1021600010B103685B6898470025244E244F56F849
:10217000352001A839465FFA85F8FFF763FB019B1C
:10218000A0680022A360019210B103685B689847C1
:10219000019810B103685B689847A368DBB141F20E
:1021A000883084F88C8001F071FF2046FFF7E2FC54
:1021B0001E2001F06BFF2046FFF70AFD054680B99F
:1021C00094F88C300F4856F83310FFF759F9284629
:1021D00002B0BDE8F0810135032DC8D10A48FFF7F0
:1021E0004DFC2046FFF760FF94F88C30054656F80A
:1021F000331008B90548E8E70548E6E770680008C5
:1022000000250020D46700084A680008FE6700081F
:10221000286800082DE9F041044688B00F461646AC
:10222000FFF71CFF2046FFF70FFF0025C722A0681D
:102230004FF48073079503A9CDE90323CDE9055534
:1022400003685B699847A0682A4629460368009599
:10225000D3F810802B46C047054630B92046FFF71B
:1022600011FF284608B0BDE8F081E36E3B60236FA4
:102270003360F3E72DE9F041002588B01F4604469E
:102280000E460E9B00F1400CA8463D60016B81B1EB
:10229000A9420ED391420CD8B6FBF1FE01FB1E61A0
:1022A00039B9416B90F82C800F9D1960816B2960C2
:1022B000154610306045E9D16DB3AB1962699342A0
:1022C00029D82046FFF7CAFE2046FFF7BDFE4FF48F
:1022D0001453A06803A9CDF80C80CDE9043600267C
:1022E000CDE9066603685B699847A06832463146C7
:1022F00003680096D3F810803346C0470646204650
:102300002EB9FFF7BFFE304608B0BDE8F081FFF7F9
:10231000B9FE3D60F7E70026F5E700002DE9F04142
:102320008669054688B00F46B3429046B1FBF6FC7D
:1023300006FB1C1C28BF3346A6EB0C0C00269C4554
:10234000644628BF1C46FFF789FE2846FFF77CFE3F
:102350000222A86803A9164B0597CDE90323CDE90E
:10236000066603685B699847A86822464146036889
:1023700000961F693346B847064628462EB9FFF730
:1023800081FE304608B0BDE8F081FFF77BFE0E9B72
:102390001C60AB6FAA696343B3FBF2F30F9A13603F
:1023A000EA6F109B5443AA69B4FBF2F41C60E8E79F
:1023B000002500012DE9F04FCE18436989B004468D
:1023C0009E420F46904634D83D464FF00009DFF854
:1023D00070A0FFF739FEAE422FD9A6EB050B94F89B
:1023E000803094F8882003A9BBF5806F039394F89C
:1023F000813028BF4FF4806B012AA06808BF03F129
:10240000FF33CDF810A0CDE90559079303685B6948
:102410009847A068A8EB07030268CDF800B02B44EA
:10242000D2F810B000221146D84718B105F58065E2
:10243000D1E7002009B0BDE8F08F0120FAE700BF26
:1024400000ED0003F0B5044689B00E46FFF7FCFD31
:1024500094F887502DB194F889302BB1012B1DD001
:102460000025284609B0F0BD94F880200392A522EB
:1024700006921A4ACDE9042394F88130A06803A992
:10248000079303685B699847A068314603689B69B6
:1024900098470546642001F0F9FDE2E72046002751
:1024A000FFF7DCFD2046FFF7CFFD082381228521C1
:1024B00020460097FFF794FD054618B92046FFF720
:1024C000E1FDCEE794F8803006970393044BCDE905
:1024D000043794F88130013BD0E700BF00ED0003E2
:1024E00000ED0013014B024A1A60704700250020DE
:1024F000C0670008036800211B68184703790BB107
:10250000002202711846704703685B681847000094
:1025100003791BB9012303711846704700207047E7
:102520007047000010B5044604F012F8204610BDB4
:1025300030B50A44084D91420DD011F8013B584086
:10254000082340F30004013B2C4013F0FF0384EA0E
:102550005000F6D1EFE730BD2083B8EDF0B500F1C3
:102560000B0423460D46B1FBF2F102FB115707F1B4
:102570003006392EC8BF07F13706954203F8016DC2
:10258000F0D2421EE11A13F8015B9C4202F8015F8F
:10259000F9D10844F0BD00002DE9F04F804687B026
:1025A00015464FF000090C4614F8013B002B3BD0B8
:1025B000252B08D0D8F800201946404609F101091A
:1025C000D268904749E14B782D2B06BF8C1C012324
:1025D0000023019323782B2B06BF0134012700270A
:1025E00094F800A0BAF1300F0CBF01344FF0200A6C
:1025F00023782A2B1CD16178023455F804BB2E298C
:1026000043D1217881B12A2921D0661C0020A1F173
:1026100030023446D2B2092A1DD80A2316F8011B0B
:1026200003FB00200029F2D1484607B0BDE8F08F37
:102630004FF0000B14F8011B0029F5D0A1F1300276
:10264000D2B2092ADBD80A2303FB0B2BF2E761780D
:10265000023455F8040B01F0DF024C2A17D121781F
:102660000029E1D0782904F101041FD8622900F281
:10267000008158291AD84E2900F23081442900F0EF
:102680009180492900F08E8010E00020E3E7A1F15D
:1026900041027829D2B209D862290BD8582905D825
:1026A0004E293BD8442978D0492976D02E468DF83A
:1026B0000C1056E0A1F16306152EF7D80FF2040CAA
:1026C0005CF826F0552700089B270008AD26000877
:1026D000AD260008AD260008AD2600089B2700089F
:1026E000AD260008AD260008AD260008AD2600087E
:1026F000AD2600082B28000819290008AD2600087F
:10270000AD2600086B270008AD2600081529000833
:10271000AD260008AD26000819290008A1F14F02D6
:10272000092AC3D801A050F822F000BF2B280008C6
:1027300019290008AD260008AD260008AD260008BE
:10274000AD26000815290008AD260008AD260008B2
:10275000192900082E464FF0200A56F8042B8DF850
:102760000C2003AD0DF10D002BE02E4647F6FF7255
:102770006A4B56F8045B002808BF1046002D08BFBE
:102780001D462A462F18104612F8011B11B1B91A1E
:102790000029F8DA4FF0200A13E02E46192A56F8DD
:1027A000041B02D82E4656F8041B002936DA2D22C7
:1027B00049428DF80C200DF10D000A2203ADFFF700
:1027C000CDFE471B0199ABEB070323EAE372002917
:1027D00045D1002BC2F1000B1EDD29782D2901D037
:1027E0002B290DD1BAF1300F0AD1D8F8003040466C
:1027F000019209F10109DB68013F98470135019A0F
:10280000D8F80030514640460192DB6898471BF1EA
:10281000010B019AF4D191443B4615E01FB12B22E4
:102820008DF80C20C7E703A8C7E708222E4603A8A7
:1028300056F8041BC2E7D8F80020404615F8011BE3
:10284000D26801939047019B013BF4D5002FA8BFAC
:10285000B9445D462DB9D94435462146A3E6934691
:10286000DAE7D8F8003051464046013DDB6898472A
:10287000F0E7A1F16302152A3FF618AF01A353F860
:1028800022F000BF55270008A5270008AD26000844
:10289000AD260008AD260008AD260008A5270008D3
:1028A000AD260008AD260008AD260008AD260008BC
:1028B000AD2600082B28000819290008AD260008BD
:1028C000AD2600086B270008AD2600081529000872
:1028D000AD260008AD26000819290008A1F14F0215
:1028E000092A3FF6E3AE01A353F822F02B28000893
:1028F00019290008AD260008AD260008AD260008FD
:10290000AD26000815290008AD260008AD260008F0
:10291000192900080A2289E7102287E7F0680008D1
:10292000F0B5054687B016461F460C4689B14A1ECB
:102930000023294601A800F053F83A46314601A881
:10294000FFF72AFE049BA3423CBF0022EA5407B0D3
:10295000F0BD0A46ECE70000D0E902239A421FBF0F
:102960004268D154C36801331ABFC36000206FF0BE
:1029700001007047D0E903239A421FBF4268D25C2E
:102980000133036114BF10466FF00100704700006F
:1029900038B504460846D4E903315B1A934228BF90
:1029A00013461D4663682A461944FEF797FD2369BE
:1029B00028462B44236138BD38B50446D0E902309F
:1029C0001B1A934228BF13461D4663682A461844C3
:1029D000FEF784FDE36828462B44E36038BD000021
:1029E00010B5C0E90223034C0023C0E90041036194
:1029F00010BD00BFF868000838B5836904460D466D
:102A00005B695A0118D543681B682BB10522027017
:102A100098472378052B01D102232370202383F3C9
:102A20001188002104F1080001F04AFB002383F320
:102A30001188E06902F07AFAEB0704D50248BDE894
:102A4000384001F0B3BA38BD0C69000810B5044C29
:102A5000204601F039F8034A0023C4E9062310BDDB
:102A6000082500200050005210B503780446012BC1
:102A700017D1104B984214D102460F49102002F092
:102A800021FA0E4BE061D3F8D42042F48042C3F81F
:102A9000D420D3F8FC2042F48042C3F8FC20D3F8C1
:102AA000FC306268A36992685A60054A1A601B226A
:102AB000DA6010BD08250020F929000800440258FA
:102AC0001500020183691B2210B5DA60D1E90020EC
:102AD00012F44C4406D192011C61D86102F44042C8
:102AE0005A6110BD0024104312F4406F1C61CC6881
:102AF000DC61586101D08A689A619A689206FCD4B8
:102B0000EFE7000030B584691B25C069E560006807
:102B1000836104F12003C36102234261013A03612E
:102B20004623C36016238362CB682261E361D1E947
:102B30000023134312F4406F636101D08B68A361DB
:102B4000C36843F00103C36030BD000030B5D0E975
:102B50000640006804F120058561C36108234261D5
:102B6000013A036146230D69C36016238362CB6873
:102B70002261E361D1E90023134312F4406F43EA79
:102B8000854343F08063636101D08B68A361C368B0
:102B900043F00103C36030BD8069036823F0040380
:102BA00010B5036000230361C3618361D1E9004371
:102BB0000969234343EA814343F04063436112B10F
:102BC0004FF01043136010BD83691A6842F002028F
:102BD0001A601A689207FCD41A6842F004021A605C
:102BE0007047000083691B2210B5DA6004465B69F8
:102BF0005B011AD443681B682BB105220270984709
:102C00002378052B01D102232370202383F311881D
:102C1000002104F1080001F053FA002383F3118826
:102C2000E069BDE8104002F081B910BD0268436858
:102C30001143016003B1184770470000024A13684E
:102C400043F0C0031360704700100140024A13684C
:102C500043F0C003136070470078004037B51A4C4A
:102C60001A4D204600F0C0FA04F11400009400232D
:102C70004FF40072164900F081F94FF400721549C3
:102C800004F138000094144B00F0FAF9134BC4E936
:102C90001735134C204600F0A7FA04F11400002366
:102CA0004FF400720F49009400F068F90E4B4FF496
:102CB00000720E4904F13800009400F0E1F90C4B69
:102CC000C4E9173503B030BD2825002000E1F50523
:102CD00000260020002A00203D2C000800100140A2
:102CE00094250020002800204D2C0008002C0020F6
:102CF00000780040037C30B52D4C002918BF0C46ED
:102D0000012B11D12B4B98423BD12B4BD3F8F02008
:102D100042F01002C3F8F020D3F8182142F010025C
:102D2000C3F81821D3F818312268036EC16D03EB84
:102D300052038466B3FBF2F36268150442BF23F0CA
:102D4000070503F0070343EA4503CB60A36843F09C
:102D500040034B60E36843F001038B6042F49673D9
:102D600043F001030B604FF0FF330B62510505D5B3
:102D700012F0102218D0B2F1805F17D080F86430C2
:102D800030BD0E4B9842CFD10B4BD3F8E82042F028
:102D90008042C3F8E820D3F8102142F08042C3F803
:102DA0001021D3F81031BFE77F23E7E73F23E5E7A2
:102DB0001C690008282500200044025894250020A2
:102DC0002DE9F047C66D05463768F469210734627E
:102DD00019D014F0080118BF8021E20748BF41F064
:102DE0002001A3074FF0200348BF41F040016007D6
:102DF00048BF41F4807183F31188281DFFF716FF47
:102E0000002383F31188E2050AD5202383F3118878
:102E10004FF40071281DFFF709FF002383F3118889
:102E20004FF020094FF0000A14F0200838D13B067B
:102E300016D54FF0200905F1380A200610D589F380
:102E40001188504600F050F9002836DA0821281D74
:102E5000FFF7ECFE27F080033360002383F3118833
:102E6000790614D5620612D5202383F31188D5E99B
:102E700013239A4208D12B6C33B127F0400710215D
:102E8000281DFFF7D3FE3760002383F31188E30684
:102E900018D5AA6E1369ABB15069BDE8F047184761
:102EA00089F31188736A284695F86410194000F078
:102EB000B5F98AF31188F469B6E7B06288F311882E
:102EC000F469BAE7BDE8F087F8B5154682680446AC
:102ED0000B46AA4200D28568A1692669761AB542D6
:102EE0000BD218462A46FEF7F9FAA3692B44A361D0
:102EF0002846A3685B1BA360F8BD0CD9AF1B18461E
:102F00003246FEF7EBFA3A46E1683044FEF7E6FA5D
:102F1000E3683B44EBE718462A46FEF7DFFAE3682E
:102F2000E5E7000083689342F7B50446154600D2F2
:102F30008568D4E90460361AB5420BD22A46FEF7FA
:102F4000CDFA63692B4463612846A3685B1BA360C9
:102F500003B0F0BD0DD93246AF1B0191FEF7BEFAAA
:102F600001993A46E0683144FEF7B8FAE3683B4419
:102F7000E9E72A46FEF7B2FAE368E4E710B50A4447
:102F80000024C361029B8460C16002610362C0E9E6
:102F90000000C0E9051110BD08B5D0E90532934223
:102FA00001D1826882B98268013282605A1C426112
:102FB00019700021D0E904329A4224BFC3684361EA
:102FC00001F098F8002008BD4FF0FF30FBE700004B
:102FD00070B5202304460E4683F31188A568A5B179
:102FE000A368A269013BA360531CA3611578226901
:102FF000934224BFE368A361E3690BB1204698477D
:10300000002383F31188284607E03146204601F06B
:1030100061F80028E2DA85F3118870BD2DE9F74FD9
:1030200004460E4617469846D0F81C904FF0200AEA
:103030008AF311884FF0000B154665B12A463146D8
:103040002046FFF741FF034660B94146204601F0A4
:1030500041F80028F1D0002383F31188781B03B0D6
:10306000BDE8F08FB9F1000F03D001902046C847AA
:10307000019B8BF31188ED1A1E448AF31188DCE75B
:10308000C160C361009B82600362C0E90511114405
:10309000C0E9000001617047F8B504460D461646C8
:1030A000202383F31188A768A7B1A368013BA3601D
:1030B00063695A1C62611D70D4E904329A4224BFCC
:1030C000E3686361E3690BB120469847002080F311
:1030D000118807E03146204600F0FCFF0028E2DAC4
:1030E00087F31188F8BD0000D0E9052310B59A4296
:1030F00001D182687AB982680021013282605A1C4B
:1031000082611C7803699A4224BFC368836100F01E
:10311000F1FF204610BD4FF0FF30FBE72DE9F74FE0
:1031200004460E4617469846D0F81C904FF0200AE9
:103130008AF311884FF0000B154665B12A463146D7
:103140002046FFF7EFFE034660B94146204600F0F7
:10315000C1FF0028F1D0002383F31188781B03B04E
:10316000BDE8F08FB9F1000F03D001902046C847A9
:10317000019B8BF31188ED1A1E448AF31188DCE75A
:10318000026843681143016003B1184770470000AB
:103190001430FFF743BF00004FF0FF331430FFF748
:1031A0003DBF00003830FFF7B9BF00004FF0FF33DC
:1031B0003830FFF7B3BF00001430FFF709BF00003D
:1031C0004FF0FF311430FFF703BF00003830FFF736
:1031D00063BF00004FF0FF323830FFF75DBF0000E3
:1031E00000207047FFF73ABD044B036000234360A3
:1031F000C0E9023301230374704700BF346900083B
:1032000010B52023044683F31188FFF773FD0223D2
:103210002374002383F3118810BD000038B5C369FF
:1032200004460D461BB904210844FFF7A9FF2946AF
:1032300004F11400FFF7B0FE002806DA201D4FF459
:103240008061BDE83840FFF79BBF38BD0268436826
:103250001143016003B118477047000013B5406B7C
:1032600000F58054D4F8A4381A681178042914D1D0
:10327000017C022911D11979012312898B40134253
:103280000BD101A94C3002F09DFCD4F8A4480246B1
:10329000019B2179206800F0DFF902B010BD000029
:1032A000143002F01FBC00004FF0FF33143002F066
:1032B00019BC00004C3002F0F1BC00004FF0FF33AD
:1032C0004C3002F0EBBC0000143002F0EDBB00000B
:1032D0004FF0FF31143002F0E7BB00004C3002F039
:1032E000BDBC00004FF0FF324C3002F0B7BC000014
:1032F0000020704710B500F58054D4F8A4381A683F
:103300001178042917D1017C022914D1597901239C
:1033100052898B4013420ED1143002F07FFB0246DB
:1033200048B1D4F8A4484FF4407361792068BDE8EF
:10333000104000F07FB910BD406BFFF7DBBF00000D
:10334000704700007FB5124B012504260446036038
:103350000023057400F1840243602946C0E902336A
:103360000C4B0290143001934FF44073009602F01E
:1033700031FB094B04F69442294604F14C000294B7
:10338000CDE900634FF4407302F0F8FB04B070BD68
:103390005C690008393300085D3200080A682023A0
:1033A00083F311880B790B3342F823004B791333E5
:1033B00042F823008B7913B10B3342F8230000F558
:1033C0008053C3F8A41802230374002383F31188E5
:1033D0007047000038B5037F044613B190F85430AD
:1033E000ABB90125201D0221FFF730FF04F11400C5
:1033F0006FF00101257700F089FE04F14C0084F89C
:1034000054506FF00101BDE8384000F07FBE38BD78
:1034100010B5012104460430FFF718FF002323777D
:1034200084F8543010BD000038B50446002514302F
:1034300002F0E8FA04F14C00257702F0B7FB201DFA
:1034400084F854500121FFF701FF2046BDE83840C1
:10345000FFF750BF90F8803003F06003202B06D1B7
:1034600090F881200023212A03D81F2A06D80020A3
:103470007047222AFBD1C0E91D3303E0034A4267AB
:1034800007228267C3670120704700BF38220020EF
:1034900037B500F58055D5F8A4381A681178042995
:1034A0001AD1017C022917D11979012312898B4085
:1034B000134211D100F14C04204602F037FC58B100
:1034C00001A9204602F07EFBD5F8A4480246019BE4
:1034D0002179206800F0C0F803B030BD01F10B0382
:1034E000F0B550F8236085B004460D46FEB12023A8
:1034F00083F3118804EB8507301D0821FFF7A6FE32
:10350000FB6806F14C005B691B681BB1019002F07F
:1035100067FB019803A902F055FB024648B1039BE3
:103520002946204600F098F8002383F3118805B05F
:10353000F0BDFB685A691268002AF5D01B8A013B6E
:103540001340F1D104F18002EAE70000133138B5ED
:1035500050F82140ECB1202383F3118804F5805307
:10356000D3F8A4281368527903EB8203DB689B69C4
:103570005D6845B104216018FFF768FE294604F133
:10358000140002F055FA2046FFF7B4FE002383F33F
:10359000118838BD7047000001F048BD012340226A
:1035A000002110B5044600F8303BFDF7C9FF0023A9
:1035B000C4E9013310BD000010B52023044683F395
:1035C00011882422416000210C30FDF7B9FF20460C
:1035D00001F04EFD02232370002383F3118810BDF8
:1035E00070B500EB8103054650690E461446DA605B
:1035F00018B110220021FDF7A3FFA06918B1102215
:103600000021FDF79DFF31462846BDE8704001F0DE
:1036100041BE000083682022002103F0011310B591
:10362000044683601030FDF78BFF2046BDE8104054
:1036300001F0BCBEF0B4012500EB810447898D4048
:10364000E4683D43A469458123600023A260636070
:10365000F0BC01F0D9BE0000F0B4012500EB8104FC
:1036600007898D40E4683D43646905812360002338
:10367000A2606360F0BC01F04FBF000070B5022390
:1036800000250446242203702946C0F888500C30D7
:1036900040F8045CFDF754FF204684F8705001F0B8
:1036A0008DFD63681B6823B129462046BDE8704044
:1036B000184770BD037880F88C3005230370436889
:1036C0001B6810B504460BB1042198470023A36082
:1036D00010BD000090F88C20436802701B680BB18D
:1036E000052118477047000070B590F87030044607
:1036F00013B1002380F8703004F18002204601F0FD
:1037000079FE63689B68B3B994F8803013F0600564
:1037100035D00021204602F023F90021204602F096
:1037200013F963681B6813B10621204698470623E6
:1037300084F8703070BD204698470028E4D0B4F873
:103740008630A26F9A4288BFA36794F98030A56F34
:10375000002B4FF0200380F20381002D00F0F28057
:10376000092284F8702083F3118800212046D4E9CF
:103770001D23FFF771FF002383F31188DAE794F824
:10378000812003F07F0343EA022340F20232934296
:1037900000F0C58021D8B3F5807F48D00DD8012B2B
:1037A0003FD0022B00F09380002BB2D104F18802AD
:1037B00062670222A267E367C1E7B3F5817F00F089
:1037C0009B80B3F5407FA4D194F88230012BA0D127
:1037D000B4F8883043F0020332E0B3F5006F4DD007
:1037E00017D8B3F5A06F31D0A3F5C063012B90D8E3
:1037F0006368204694F882205E6894F88310B4F8D9
:103800008430B047002884D0436863670368A367A7
:103810001AE0B3F5106F36D040F6024293427FF4BF
:1038200078AF5C4B63670223A3670023C3E794F878
:103830008230012B7FF46DAFB4F8883023F002039F
:10384000A4F88830C4E91D55E56778E7B4F88030FE
:10385000B3F5A06F0ED194F88230204684F88A30F8
:1038600001F00AFD63681B6813B1012120469847E7
:10387000032323700023C4E91D339CE704F18B0369
:1038800063670123C3E72378042B10D1202383F33C
:1038900011882046FFF7BEFE85F311880321636877
:1038A00084F88B5021701B680BB12046984794F820
:1038B0008230002BDED084F88B30042323706368C1
:1038C0001B68002BD6D0022120469847D2E794F8F7
:1038D000843020461D0603F00F010AD501F07CFD5F
:1038E000012804D002287FF414AF2B4B9AE72B4B0E
:1038F00098E701F063FDF3E794F88230002B7FF442
:1039000008AF94F8843013F00F01B3D01A062046A4
:1039100002D502F03DF8ADE702F02EF8AAE794F8E0
:103920008230002B7FF4F5AE94F8843013F00F0151
:10393000A0D01B06204602D502F012F89AE702F04A
:1039400003F897E7142284F8702083F311882B463C
:103950002A4629462046FFF76DFE85F31188E9E6E1
:103960005DB1152284F8702083F311880021204670
:10397000D4E91D23FFF75EFEFDE60B2284F87020DC
:1039800083F311882B462A4629462046FFF764FE1A
:10399000E3E700BF8C6900088469000888690008B3
:1039A00038B590F870300446002B3ED0063BDAB2B2
:1039B0000F2A34D80F2B32D8DFE803F03731310823
:1039C000223231313131313131313737856FB0F811
:1039D00086309D4214D2C3681B8AB5FBF3F203FB09
:1039E00012556DB9202383F311882B462A462946A8
:1039F000FFF732FE85F311880A2384F870300EE059
:103A0000142384F87030202383F311880023204688
:103A10001A461946FFF70EFE002383F3118838BDBE
:103A2000C36F03B198470023E7E70021204601F068
:103A300097FF0021204601F087FF63681B6813B1E0
:103A40000621204698470623D7E7000010B590F8D6
:103A500070300446142B29D017D8062B05D001D876
:103A60001BB110BD093B022BFBD80021204601F001
:103A700077FF0021204601F067FF63681B6813B1E0
:103A8000062120469847062319E0152BE9D10B2380
:103A900080F87030202383F3118800231A461946DA
:103AA000FFF7DAFD002383F31188DAE7C3689B6927
:103AB0005B68002BD5D1C36F03B19847002384F80E
:103AC0007030CEE7FEF7C2BF012100230170C0E9CC
:103AD00001330C3000F008BA10B52023044683F3FC
:103AE00011884160FEF7C0FF02232370002383F397
:103AF000118810BD10B52023044683F311880323D9
:103B000004F8083BFEF7DEFF4FF0FF31204600F0DF
:103B1000C9FA002383F31188C01A18BF012010BD11
:103B200038B50446202585F31188032504F8085B81
:103B3000FEF7E8FF4FF0FF31204600F0B3FA002314
:103B400083F31188C01A18BF012038BD38B5044668
:103B5000202585F31188042504F8085BFEF7F6FF9D
:103B60004FF0FF31204600F09DFA002383F31188C7
:103B7000C01A18BF012038BD10B52023044683F3B6
:103B80001188FFF709F806232370002383F31188B7
:103B900010BD000010B52023044683F31188FFF701
:103BA00013F802232370002383F3118810BD000053
:103BB0000C3000F0B5B900000C3000F0BBB90000CB
:103BC00004480121044B03600023C0E901330C3099
:103BD00000F08AB9002E0020E15D0008CB1D083AF4
:103BE00023F00703591A521A012110B4D2080024F5
:103BF000C0E9004384600C301C605A605DF8044BDF
:103C000000F072B92DE9F84F364ECD1D0F46002851
:103C100018BF0646082A4FEAD50538BF082206F124
:103C20000C08341D9146404600F07AF909F107016D
:103C3000C9F1000E224624686CB9404600F07AF9BA
:103C40003368CBB308224946E8009847044698B346
:103C500040E9026730E004EB010CD4F804A00CEA60
:103C60000E0C0AF10100ACF1080304EBC00098420D
:103C7000E0D9A0EB0C0CB5EBEC0F4FEAEC0BD9D86C
:103C80009C421CD204F10802AB45A3EB02024FEAAE
:103C9000E202626009D9691CED43206803EBC102AE
:103CA0005D44556043F8310022601C465F60404629
:103CB00044F8086B00F03EF92046BDE8F88FAA45AD
:103CC000216802D111602346EFE7013504EBC503FB
:103CD00044F8351003F10801401AC0105860136011
:103CE000F1E700BF002E0020F8B550F8043C044670
:103CF00050F8085CA0F1080607332F1D0C35DB08CF
:103D000040F8043C284600F00BF93B46BB421A68D9
:103D100001D09E4228D90AB1964225D244F8082CF7
:103D200054F8042C1E60013254F8081C06EBC20043
:103D3000814206D14868024444F8042C0A6844F8D9
:103D4000082C5868411C03EBC1018E4207D154F87E
:103D5000042C013202445A6054F8082C1A60284698
:103D6000BDE8F84000F0E6B81346CFE7024B00226A
:103D7000C3E900339A607047182E00200023826840
:103D80000374054B1B6899689142FBD25A68036023
:103D90004260106058607047182E002008B520233C
:103DA00083F31188027C0023052A06D8DFE802F09D
:103DB0000B050503120E426913604FF0FF33436198
:103DC000FFF7DCFF002383F3118808BD4269936885
:103DD00001339360D0E9003213605A60EDE70000D0
:103DE000002382680374054B1B6899689142FBD8D5
:103DF0005A6803604260106058607047182E0020B7
:103E0000054B196908741868026853601A601861D4
:103E100001230374FCF764BC182E00204B1C30B542
:103E2000044687B00A4D10D02B6901A8094A00F05A
:103E300089F92046FFF7E4FF049B13B101A800F0C5
:103E4000BDF92B69586907B030BDFFF7D9FFF8E716
:103E5000182E00209D3D000838B50C4D04464161E8
:103E60002B6981689A68914203D8BDE83840FFF712
:103E700085BF1846FFF7B4FF01232C610146237468
:103E80002046BDE83840FCF72BBC00BF182E0020B0
:103E9000044B1A681B6990689B68984294BF002085
:103EA00001207047182E002010B5084C23682069A7
:103EB0001A6854602260012223611A74FFF790FF90
:103EC00001462069BDE81040FCF70ABC182E00200E
:103ED00008B5FFF7DDFF18B1BDE80840FFF7E4BF04
:103EE00008BD0000FFF7E0BFC0E900008160704737
:103EF0008368013B002B10B583600DDA074C4268E4
:103F00002369586118605A60136043600520FFF709
:103F100077FF2369586910BD0020FCE7182E0020A8
:103F200008B5202383F31188FFF7E2FF002383F312
:103F3000118808BD08B5202383F3118883680133F5
:103F4000002B836007DC036800211A680260506060
:103F50001846FFF781FF002383F3118808BD000096
:103F6000FEE7000010B50E4CFFF700FF00F0DCF894
:103F700001F018FFFFF724FE80220A49204600F0D6
:103F800047F8012344F8180C037400F053FE002393
:103F900083F3118862B60448BDE8104000F058B8B9
:103FA000402E002090690008A069000808B572B68C
:103FB000034B586200F0C0FC00F08EFDFEE700BF2E
:103FC000182E002000F034B9EFF3118020B9EFF380
:103FD0000583202282F311887047000010B530B9A4
:103FE000EFF30584C4F3080414B180F3118810BD05
:103FF000FFF76EFF84F31188F9E70000034A516868
:1040000053685B1A9842FBD8704700BF001000E06D
:1040100082600222028270478368A3F17C0243F827
:104020000C2C026943F83C2C426943F8382C074AAF
:1040300043F81C2CC268A3F1180043F8102C02228C
:1040400003F8082C002203F8072C7047F906000833
:1040500010B5202383F31188FFF7DEFF002104460B
:10406000FFF7FAFE002383F31188204610BD0000FD
:10407000024B1B6958610F20FFF7C2BE182E0020AB
:10408000202383F31188FFF7F3BF000008B5014632
:10409000202383F311880820FFF7C0FE002383F359
:1040A000118808BD054B1B6921B1036058610320CD
:1040B000FFF7B4BE4FF0FF30704700BF182E00204E
:1040C00003682BB10022026018465961FFF756BE03
:1040D0007047000049B1064B42681B6918605A607E
:1040E000136043600420FFF799BE4FF0FF30704724
:1040F000182E00200368984206D01A6802605060AB
:1041000018465961FFF73ABE7047000038B50446BB
:104110000D462068844200D138BD036823605C608E
:104120004561FFF72BFEF4E7054B4FF0FF3103F13C
:104130001402C3E905220022C3E90712704700BF39
:10414000182E002070B51C4E05460C46C0E903230E
:1041500001F022FE334653F8142F9A420DD13062FB
:104160000A2C2CBF00190A302A60C5E90124C6E9CF
:104170000555BDE8704001F0F9BD316A431AE318F6
:1041800038BF1C469368A34202D9081901F0FEFD0E
:1041900073699A6894420CD85A68AC602B606A6064
:1041A00015609A685D60121B9A604FF0FF33F361EF
:1041B00070BDA41A1B68ECE7182E002038B51B4C04
:1041C000636998420DD08168D0E9003213605A606B
:1041D0000022C2609A680A449A604FF0FF33E3619C
:1041E00038BD03682246002142F8143F93425A60CA
:1041F000C16003D1BDE8384001F0C2BD9A68816852
:10420000256A0A449A6001F0C7FD6369411B9A68F8
:104210008A42E5D9AB181D1A206A092D98BF01F111
:104220000A02BDE83840104401F0B0BD182E00204D
:104230002DE9F041184C002704F11406656901F0DE
:10424000ABFD236AAA68C11A8A4215D81344D5F86F
:104250000C802362D5E9003213605A606369EF6015
:10426000B34201D101F08CFD87F311882869C04762
:10427000202383F31188E1E76169B14209D0134437
:104280001B1ABDE8F0410A2B2CBFC0180A3001F000
:104290007DBDBDE8F08100BF182E002000207047D2
:1042A000FEE70000704700004FF0FF30704700004D
:1042B00002290CD0032904D00129074818BF002087
:1042C0007047032A05D8054800EBC2007047044830
:1042D00070470020704700BF846A00084822002011
:1042E000386A000870B59AB005460846144601A918
:1042F00000F0C2F801A8FDF71BF9431C0022C6B26A
:104300005B001046C5E9003423700323023404F82F
:10431000013C01ABD1B202348E4201D81AB070BD5B
:1043200013F8011B013204F8010C04F8021CF1E738
:1043300008B5202383F311880348FFF7A9F8002369
:1043400083F3118808BD00BFD02F002090F8803083
:1043500003F01F02012A07D190F881200B2A03D114
:104360000023C0E91D3315E003F06003202B08D1C2
:10437000B0F884302BB990F88120212A03D81F2A65
:1043800004D8FFF767B8222AEBD0FAE7034A42675E
:1043900007228267C3670120704700BF3F220020C9
:1043A00007B5052917D8DFE801F0191603191920F8
:1043B000202383F31188104A01210190FFF710F99F
:1043C000019802210D4AFFF70BF90D48FFF72CF871
:1043D000002383F3118803B05DF804FB202383F3EB
:1043E00011880748FEF7F6FFF2E7202383F31188D0
:1043F0000348FFF70DF8EBE7D8690008FC690008EF
:10440000D02F002038B50C4D0C4C2A460C4904F135
:104410000800FFF767FF05F1CA0204F1100009491F
:10442000FFF760FF05F5CA7204F118000649BDE800
:104430003840FFF757BF00BFA8480020482200209F
:10444000B8690008C2690008CD69000870B5044663
:1044500008460D46FDF76CF8C6B2204601340378D5
:104460000BB9184670BD32462946FDF741F80028C1
:10447000F3D10120F6E700002DE9F84F05460C4680
:10448000FDF756F82D49C6B22846FFF7DFFF08B101
:104490000436F6B22A492846FFF7D8FF08B110368D
:1044A000F6B2632E0DD8DFF89490DFF894A0DFF811
:1044B0009C80DFF89CB0234F2E7846B92670BDE86B
:1044C000F88F29462046BDE8F84F02F0C9B8252EDE
:1044D00030D1072249462846FDF70AF870B93B68F3
:1044E00007350B3444F80B3C7B6844F8073C3B89A8
:1044F00024F8033CBB7A04F8013CDDE7082251466E
:104500002846FCF7F5FFA8B9A21C0F4B1978023218
:10451000090911F8081002F8041C13F8011B01F036
:104520000F015B4511F8081002F8031CEED1183496
:104530000835C1E7013504F8016BBDE7A46A00083E
:10454000CD690008AC6A000800E8F11FB86A0008ED
:104550000CE8F11FBFF34F8F044B1A695107FCD1D0
:10456000D3F810215207F8D1704700BF0020005245
:1045700008B50D4B1B78ABB9FFF7ECFF0B4BDA68B6
:10458000D10704D50A4A5A6002F188325A60D3F83A
:104590000C21D20706D5064AC3F8042102F188325D
:1045A000C3F8042108BD00BF064B002000200052C4
:1045B000230167454FF00063054A1968013104D1B2
:1045C00004339342F9D1012070470020704700BFA7
:1045D0000000020808B5114B1B78F3B9104B1A699B
:1045E000510703D5DA6842F04002DA60D3F81021AF
:1045F000520705D5D3F80C2142F04002C3F80C2134
:10460000FFF7A8FF064BDA6842F00102DA60D3F840
:104610000C2142F00102C3F80C2108BD064B00201A
:10462000002000524FF40030704700000120704716
:1046300008B9FFF7BFBF00207047000038B548BB7E
:10464000154CFFF7C1FCFFF785FF0546FFF790FF0C
:104650004FF0FF336361C4F814312361FFF77AFF31
:104660002423E360E36843F08003E36023695B078E
:10467000FCD4FFF76FFF4FF000604FF4003100F003
:1046800007FA2846FFF7A6FFFFF7A8FCBDE8384069
:10469000FFF790BF002038BD002000522DE9F84FF1
:1046A00040EA020305460C461746D80602D0002011
:1046B000BDE8F88F27F01F07DFF8D4B0FFF758FFE9
:1046C0002744BC4203D10120FFF784FFF0E72022FA
:1046D0002946204601F070FF10B920352034F0E75C
:1046E0002B4605F120021E68711CE0D104339A426A
:1046F000F9D1FFF769FC05F17843234AB3F5801F30
:10470000224B28BF9A4603F1040338BF9046A2F11A
:10471000080228BF9846A3F108033ABF9146DA463B
:104720009946FFF717FFC8F80060A5EB040CD9F80D
:10473000002004F11C0142F00202C9F80020221FEF
:10474000DAF8006016F00506FAD152F8043F8A4202
:104750004CF80230F4D1BFF34F8FFFF7FBFE4FF060
:10476000FF32C8F80020D9F8002022F00202C9F870
:104770000020FFF733FC20222146284601F01CFFD1
:104780000028AAD030469FE7142000521021005282
:104790001020005210B5084C237828B11BB9FFF740
:1047A000E7FE0123237010BD002BFCD02070BDE874
:1047B0001040FFF70FBF00BF064B00202DE9F74F59
:1047C0000E460546002864D011F0050763D139B9BB
:1047D000082229463046FFF715FA0446002848D13A
:1047E00008224FF00109DFF8C08006F00403DFF86B
:1047F000BCA006EA090BBBF1000F27D0D8F81410B3
:10480000C80723D409F1010908F10C08B9F1060F12
:10481000F1D18FB9224E2946F0190092FFF7F2F933
:10482000044630BB1837009A782FF4D12946FFF799
:10483000E9F90446E8B9009A29461A48FFF7E2F96F
:10484000044608BB204603B0BDE8F08FABB1D8F8F2
:10485000141011F0040FD5D01820294600FB09A030
:10486000CDE90023FFF7CEF90446DDE90023002857
:10487000C8D02A460021204608E0B107ECD5D8F878
:10488000141011F0020FE6E72A460021FCF758FE4B
:10489000D8E70446D6E71F35202225F01F05A0E7FC
:1048A000384B0020084B0020CC6A0008204B002029
:1048B0000021FFF783BF00000121FFF77FBF000049
:1048C000F8B5144D01241827134E40F2FF32002191
:1048D0000120FCF735FE07FB046001342A6955F816
:1048E0000C1FFFF77BF9062CF5D137254FF4C05488
:1048F0002046FFF7E1FF014628B122460748BDE800
:10490000F840FFF76BB9C4EBC404013D4FEAD4048F
:10491000EED1F8BDCC6A0008204B0020084B0020E7
:104920000421FFF74BBF00004843FFF7C1BF000061
:1049300008B1FFF7D9B9704738B5054D00240334E5
:10494000696855F80C0B00F0B5F8122CF7D138BD9A
:10495000CC6A000870B5104E82B0FFF735FB0546F3
:1049600001F01AFA326803469042336037BF0B4AAF
:104970000A495168146836BF0131D1E900415160DC
:104980000419284641F100010191FFF727FB204659
:10499000019902B070BD00BFB04B0020B84B0020A1
:1049A00070B5124E82B0FFF70FFB054601F0F4F927
:1049B000326803469042336037BF0D4A0C49516854
:1049C000146836BF0131D1E900415160041928460D
:1049D00041F100010191FFF701FB4FF47A720023CE
:1049E00020460199FBF764FC02B070BDB04B00207B
:1049F000B84B00200244074BD2B210B5904200D110
:104A000010BD441C00B253F8200041F8040BE0B282
:104A1000F4E700BF504000580E4B30B51C6F240423
:104A200005D41C6F1C671C6F44F400441C670A4CBF
:104A300002442368D2B243F480732360074B904250
:104A400000D130BD441C51F8045B00B243F8205043
:104A5000E0B2F4E7004402580048025850400058C1
:104A600007B5012201A90020FFF7C4FF019803B098
:104A70005DF804FB13B50446FFF7F2FFA04205D032
:104A8000012201A900200194FFF7C6FF02B010BD6A
:104A90000144BFF34F8F064B884204D3BFF34F8FBF
:104AA000BFF36F8F7047C3F85C022030F4E700BF9C
:104AB00000ED00E00144BFF34F8F064B884204D362
:104AC000BFF34F8FBFF36F8F7047C3F87002203072
:104AD000F4E700BF00ED00E07047000070B5054648
:104AE00016460C4601201021FFF71EFF2860467372
:104AF0003CB1204636B1FFF713FF2B68186000B1B8
:104B00009C6070BDFFF7D8FEF7E7000070B50E4659
:104B10001546044600B30B6843608368934210D285
:104B200013B10068FFF704FF637B28462BB1FFF742
:104B3000F7FE206020B9A06070BDFFF7BDFEF8E76A
:104B4000A560206805F11F01306021F01F01FFF70B
:104B50009FFF01202073EFE70120EDE710B5044629
:104B600040B10068884205D1606808B1FCF7B6FC26
:104B70000023237310BD000070B50E461546044691
:104B800020B38368934210D213B10068FFF7D0FEC0
:104B9000637B28462BB1FFF7C3FE206020B9A060DD
:104BA00070BDFFF789FEF8E7A560316819B12A46A4
:104BB0002068FCF793FC206805F11F01306021F0AC
:104BC0001F01FFF777FF01202073E9E70120E7E7E6
:104BD00020B103688B4204BF0023037370470000B9
:104BE00008B1002303737047034B1A681AB9034ACC
:104BF000D2F8D0241A607047C04B00200040025801
:104C000008B5FFF7F1FF024B1868C0F3806008BDDC
:104C1000C04B0020EFF30983054968334A6B22F04B
:104C200001024A6383F30988002383F311887047E4
:104C300000EF00E0202080F3118862B60D4B0E4A91
:104C4000D96821F4E0610904090C0A430B49DA60D0
:104C5000D3F8FC2042F08072C3F8FC20084AC2F866
:104C6000B01F116841F0010111601022DA7783F85A
:104C70002200704700ED00E00003FA0555CEACC5F8
:104C8000001000E0202310B583F311880E4B5B6801
:104C900013F4006314D0F1EE103AEFF309844FF0EF
:104CA0008073683CE361094BDB6B236684F30988FE
:104CB000FFF7EEF810B1064BA36110BD054BFBE703
:104CC00083F31188F9E700BF00ED00E000EF00E09A
:104CD0000B0700080E07000870B5BFF34F8FBFF336
:104CE0006F8F1A4A0021C2F85012BFF34F8FBFF3E3
:104CF0006F8F536943F400335361BFF34F8FBFF39A
:104D00006F8FC2F88410BFF34F8FD2F8803043F614
:104D1000E074C3F3C900C3F34E335B0103EA040636
:104D2000014646EA81750139C2F86052F9D2203B4A
:104D300013F1200FF2D1BFF34F8F536943F4803347
:104D40005361BFF34F8FBFF36F8F70BD00ED00E075
:104D5000FEE700000A4B0B480B4A90420BD30B4B6B
:104D6000C11EDA1C121A22F003028B4238BF002245
:104D70000021FCF7E5BB53F8041B40F8041BECE7EB
:104D80009C6D0008684E0020684E0020684E002090
:104D90007047000003681968596043680BB1806868
:104DA000184770474FF0A44310B51C68E00702D5C0
:104DB0002848FFF7EFFFA10702D52748FFF7EAFFD2
:104DC000620702D52548FFF7E5FF230702D52448EF
:104DD000FFF7E0FFE00602D52248FFF7DBFFA10660
:104DE00002D52148FFF7D6FF620602D51F48FFF71C
:104DF000D1FF230602D51E48FFF7CCFFE00502D500
:104E00001C48FFF7C7FFA10502D51B48FFF7C2FFEB
:104E1000620502D51948FFF7BDFF230502D51848E2
:104E2000FFF7B8FFE00402D51648FFF7B3FFA1046F
:104E300002D51548FFF7AEFF620402D51348FFF70D
:104E4000A9FF230402D51248FFF7A4FFBDE81040D4
:104E5000FFF718BFC84B0020D44B0020E04B0020C8
:104E6000EC4B0020F84B0020044C0020104C00209C
:104E70001C4C0020284C0020344C0020404C0020CA
:104E80004C4C0020584C0020644C0020704C0020FA
:104E90007C4C002030B5094B0021094C102007251F
:104EA000196054F8042B0138C3E90121D16003F1E2
:104EB0000C0311615560F4D130BD00BFC44B00201C
:104EC000146B00080F28F0B50AD9102806D10F235B
:104ED0000020144C01272568984203D900201DE0CA
:104EE0000346F6E707FA00F6354218D10C2335439E
:104EF00043432560181D2344C3E902120A4B204492
:104F0000D3F8D42042F00102C3F8D420D3F8FC2017
:104F100042F00102C3F8FC20D3F8FC30F0BD0130B0
:104F2000DAE700BFC44B0020004402580368D96888
:104F3000DA68C90722F03F02DA6002D51A689207E0
:104F4000FCD507225A60704770B5D0E9244300228F
:104F50004FF0FF359E6804EB42135101D3F800096E
:104F6000002805DAD3F8000940F08040C3F80009B2
:104F7000D3F8000B002805DAD3F8000B40F080408E
:104F8000C3F8000B013263189642C3F80859C3F8FE
:104F9000085BE0D24FF00113C4F81C3870BD00006C
:104FA00000EB8103D3F80CC02DE9F043DCF81420AA
:104FB0004E1CD0F89050D2F800E005EB063605EB19
:104FC0004118506870450AD30122D5F8343802FAE6
:104FD00001F123EA0101C5F83418BDE8F083AEEB16
:104FE0000003BCF81040A34228BF2346D8F8184954
:104FF000A4B2B3EB840FF0D89468A4F1040959F873
:10500000047F3760A4EB09071F44042FF7D81C4422
:10501000034494605360D4E7890141F020010161A9
:1050200003699B06FCD41220FEF7E8BF10B50A4CBA
:105030002046FEF7B3FA094BC4F89030084BC4F889
:105040009430084C2046FEF7A9FA074BC4F890307C
:10505000064BC4F8943010BD884C00200000084076
:10506000786B0008244D002000000440846B000889
:1050700070B503780546012B5DD1494BD0F89040BF
:10508000984259D1474B0E216520D3F8D82042F0E1
:105090000062C3F8D820D3F8002142F00062C3F8C0
:1050A0000021D3F80021D3F8802042F00062C3F839
:1050B0008020D3F8802022F00062C3F88020D3F84B
:1050C000803000F071FC384BE360384BC4F8003896
:1050D0000023D5F89060C4F8003EC02323604FF44D
:1050E0000413A3633369002BFCDA01230C20336122
:1050F000FEF784FF3369DB07FCD41220FEF77EFF46
:105100003369002BFCDA00262846A660FFF71CFF57
:105110006B68C4F81068DB68C4F81468C4F81C68CD
:10512000002B3AD1224BA3614FF0FF336361A36898
:1051300043F00103A36070BD1E4B9842C8D1194BC8
:105140000E214D20D3F8D82042F00072C3F8D820A9
:10515000D3F8002142F00072C3F80021D3F80021F7
:10516000D3F8802042F00072C3F88020D3F880206A
:1051700022F00072C3F88020D3F88020D3F8D82022
:1051800022F08062C3F8D820D3F8002122F0806298
:10519000C3F80021D3F8003193E7074BC3E700BF02
:1051A000884C0020004402584014004003002002B4
:1051B000003C30C0244D0020083C30C0F8B5D0F889
:1051C0009040054600214FF000662046FFF724FF7F
:1051D000D5F8941000234FF001128F684FF0FF3084
:1051E000C4F83438C4F81C2804EB431201339F423E
:1051F000C2F80069C2F8006BC2F80809C2F8080BCF
:10520000F2D20B68D5F89020C5F89830636210236D
:105210001361166916F01006FBD11220FEF7EEFEA0
:10522000D4F8003823F4FE63C4F80038A36943F4CB
:10523000402343F01003A3610923C4F81038C4F8D5
:1052400014380B4BEB604FF0C043C4F8103B094BD4
:10525000C4F8003BC4F81069C4F80039D5F8983098
:1052600003F1100243F48013C5F89820A362F8BD3F
:10527000546B000840800010D0F8902090F88A10FD
:10528000D2F8003823F4FE6343EA0113C2F8003871
:10529000704700002DE9F84300EB8103D0F89050EF
:1052A0000C468046DA680FFA81F94801166806F064
:1052B0000306731E022B05EB41134FF0000194BF50
:1052C000B604384EC3F8101B4FF0010104F110036F
:1052D00098BF06F1805601FA03F3916998BF06F56D
:1052E000004600293AD0578A04F158013743490152
:1052F0006F50D5F81C180B430021C5F81C382B182B
:105300000127C3F81019A7405369611E9BB3138A84
:10531000928B9B08012A88BF5343D8F8982098188D
:1053200042EA034301F140022146C8F898002846AA
:1053300005EB82025360FFF76FFE08EB8900C3683C
:105340001B8A43EA845348341E4364012E51D5F826
:105350001C381F43C5F81C78BDE8F88305EB4917D6
:10536000D7F8001B21F40041C7F8001BD5F81C1822
:1053700021EA0303C0E704F13F030B4A2846214614
:1053800005EB83035A60FFF747FE05EB4910D0F8A1
:10539000003923F40043C0F80039D5F81C3823EA5B
:1053A0000707D7E70080001000040002D0F894201F
:1053B0001268C0F89820FFF7C7BD00005831D0F838
:1053C000903049015B5813F4004004D013F4001FDF
:1053D0000CBF0220012070474831D0F890304901BD
:1053E0005B5813F4004004D013F4001F0CBF0220DC
:1053F0000120704700EB8101CB68196A0B681360CC
:105400004B6853607047000000EB810330B5DD68E6
:10541000AA691368D36019B9402B84BF4023136075
:105420006B8A1468D0F890201C4402EB4110013CB8
:1054300009B2B4FBF3F46343033323F0030343EAF9
:10544000C44343F0C043C0F8103B2B6803F0030390
:10545000012B0ED1D2F8083802EB411013F4807FF3
:10546000D0F8003B14BF43F0805343F00053C0F822
:10547000003B02EB4112D2F8003B43F00443C2F878
:10548000003B30BD2DE9F041D0F8906005460C4658
:1054900006EB4113D3F8087B3A07C3F8087B08D51D
:1054A000D6F814381B0704D500EB8103DB685B6872
:1054B0009847FA071FD5D6F81438DB071BD505EB3C
:1054C0008403D968CCB98B69488A5A68B2FBF0F674
:1054D00000FB16228AB91868DA6890420DD2121AB7
:1054E000C3E90024202383F3118821462846FFF7CF
:1054F0008BFF84F31188BDE8F081012303FA04F2E5
:105500006B8923EA02036B81CB68002BF3D0214621
:105510002846BDE8F041184700EB81034A0170B509
:10552000DD68D0F890306C692668E66056BB1A4496
:105530004FF40020C2F810092A6802F00302012A81
:105540000AB20ED1D3F8080803EB421410F4807F9E
:10555000D4F8000914BF40F0805040F00050C4F867
:10556000000903EB4212D2F8000940F00440C2F8EF
:1055700000090122D3F8340802FA01F10143C3F80B
:10558000341870BD19B9402E84BF402020602068B7
:105590001A442E8A8419013CB4FBF6F440EAC44054
:1055A00040F00050C6E700002DE9F041D0F89060CF
:1055B00004460D4606EB4113D3F80879C3F8087981
:1055C000FB071CD5D6F81038DA0718D500EB810395
:1055D000D3F80CC0DCF81430D3F800E0DA68964554
:1055E0001BD2A2EB0E024FF000081A60C3F8048031
:1055F000202383F31188FFF78FFF88F311883B0680
:1056000018D50123D6F83428AB40134212D02946CE
:105610002046BDE8F041FFF7C3BC012303FA01F2C5
:10562000038923EA02030381DCF80830002BE6D06B
:105630009847E4E7BDE8F0812DE9F84FD0F89050A5
:1056400004466E69AB691E4016F480586E6103D043
:10565000BDE8F84FFEF712B8002E12DAD5F8003E7A
:105660009F0705D0D5F8003E23F00303C5F8003EA0
:10567000D5F80438204623F00103C5F80438FEF7B6
:1056800029F8300505D52046FFF75EFC2046FEF7D9
:1056900011F8B1040CD5D5F8083813F0060FEB68F3
:1056A00023F470530CBF43F4105343F4A053EB6046
:1056B000320704D56368DB680BB120469847F302D4
:1056C00000F1BA80B70226D5D4F8909000274FF0A9
:1056D000010A09EB4712D2F8003B03F44023B3F56B
:1056E000802F11D1D2F8003B002B0DDA62890AFA23
:1056F00007F322EA0303638104EB8703DB68DB68BB
:1057000013B13946204698470137D4F89430FFB298
:105710009B689F42DDD9F00619D5D4F89000026A43
:10572000C2F30A1702F00F0302F4F012B2F5802F51
:1057300000F0CC80B2F5402F09D104EB83030022A6
:1057400000F58050DB681B6A974240F0B28030035E
:10575000D5F8185835D5E90303D500212046FFF7C1
:1057600091FEAA0303D501212046FFF78BFE6B03B0
:1057700003D502212046FFF785FE2F0303D5032121
:105780002046FFF77FFEE80203D504212046FFF7FD
:1057900079FEA90203D505212046FFF773FE6A02B0
:1057A00003D506212046FFF76DFE2B0203D5072106
:1057B0002046FFF767FEEF0103D508212046FFF7DB
:1057C00061FE700340F1A980E90703D5002120465E
:1057D000FFF7EAFEAA0703D501212046FFF7E4FE02
:1057E0006B0703D502212046FFF7DEFE2F0703D506
:1057F00003212046FFF7D8FEEE0603D504212046FC
:10580000FFF7D2FEA80603D505212046FFF7CCFE00
:10581000690603D506212046FFF7C6FE2A0603D5F2
:1058200007212046FFF7C0FEEB0576D5204608216C
:10583000BDE8F84FFFF7B8BED4F8909000274FF0BE
:10584000010AD4F894305FFA87FB9B689B453FF6CA
:1058500039AF09EB4B13D3F8002902F44022B2F51B
:10586000802F24D1D3F80029002A20DAD3F8002988
:1058700042F09042C3F80029D3F80029002AFBDB4C
:105880005946D4F89000FFF7C7FB22890AFA0BF3B8
:1058900022EA0303238104EB8B03DB689B6813B1CB
:1058A00059462046984759462046FFF779FB01376D
:1058B000C7E7910701D1D0F80080072A02F1010261
:1058C0009CBF03F8018B4FEA18283DE704EB8303E4
:1058D00000F58050DA68D2F818C0DCF80820DCE95E
:1058E000001CA1EB0C0C00218F4208D1DB689B69E6
:1058F0009A683A449A605A683A445A6027E711F025
:10590000030F01D1D0F800808C4501F1010184BF63
:1059100002F8018B4FEA1828E6E7BDE8F88F00008F
:1059200008B50348FFF788FEBDE80840FFF7AAB9AD
:10593000884C002008B50348FFF77EFEBDE808400C
:10594000FFF7A0B9244D0020D0F8903003EB4111AF
:10595000D1F8003B43F40013C1F8003B704700004E
:10596000D0F8903003EB4111D1F8003943F4001323
:10597000C1F8003970470000D0F8903003EB4111B6
:10598000D1F8003B23F40013C1F8003B704700003E
:10599000D0F8903003EB4111D1F8003923F4001313
:1059A000C1F8003970470000090100F1604301228D
:1059B00003F56143C9B283F8001300F01F039A4056
:1059C00043099B0003F1604303F56143C3F8802161
:1059D0001A60704730B50433039C0172002104FB48
:1059E0000325C160C0E90653049B0363059BC0E91E
:1059F0000000C0E90422C0E90842C0E90A1143637B
:105A000030BD00000022416AC260C0E90411C0E953
:105A10000A226FF00101FEF779BB0000D0E90432E1
:105A2000934201D1C2680AB9181D7047002070471F
:105A3000036919600021C2680132C260C26913445F
:105A400082699342036124BF436A0361FEF752BB3C
:105A500038B504460D46E3683BB162690020131D6A
:105A60001268A3621344E36207E0237A33B929463C
:105A70002046FEF72FFB0028EDDA38BD6FF001005D
:105A8000FBE70000C368C269013BC360436913447C
:105A900082699342436124BF436A43610023836266
:105AA000036B03B11847704770B52023044683F396
:105AB0001188866A3EB9FFF7CBFF054618B186F319
:105AC0001188284670BDA36AE26A13F8015B93420D
:105AD000A36202D32046FFF7D5FF002383F311888A
:105AE000EFE700002DE9F84F04460E4617469846AA
:105AF0004FF0200989F311880025AA46D4F828B070
:105B0000BBF1000F09D141462046FFF7A1FF20B1AC
:105B10008BF311882846BDE8F88FD4E90A12A7EB69
:105B2000050B521A934528BF9346BBF1400F1BD972
:105B3000334601F1400251F8040B914243F8040B43
:105B4000F9D1A36A403640354033A362D4E90A2331
:105B50009A4202D32046FFF795FF8AF31188BD428F
:105B6000D8D289F31188C9E730465A46FBF7B6FC0C
:105B7000A36A5E445D445B44A362E7E710B5029C00
:105B80000433017204FB0321C460C0E9061300233F
:105B9000C0E90A33039B0363049BC0E90000C0E92A
:105BA0000422C0E90842436310BD0000026A6FF09E
:105BB0000101C260426AC0E904220022C0E90A224F
:105BC000FEF7A4BAD0E904239A4201D1C26822B9EF
:105BD000184650F8043B0B607047002070470000E7
:105BE000C3680021C2690133C360436913448269F9
:105BF0009342436124BF436A4361FEF77BBA0000CE
:105C000038B504460D46E3683BB1236900201A1DF0
:105C1000A262E2691344E36207E0237A33B92946BA
:105C20002046FEF757FA0028EDDA38BD6FF0010084
:105C3000FBE7000003691960C268013AC260C269EB
:105C4000134482699342036124BF436A03610023C2
:105C50008362036B03B118477047000070B52023BF
:105C60000D460446114683F31188866A2EB9FFF764
:105C7000C7FF10B186F3118870BDA36A1D70A36AB7
:105C8000E26A01339342A36204D3E16920460439F6
:105C9000FFF7D0FF002080F31188EDE72DE9F84FE2
:105CA00004460D46904699464FF0200A8AF3118823
:105CB0000026B346A76A4FB949462046FFF7A0FF22
:105CC00020B187F311883046BDE8F88FD4E90A0780
:105CD0003A1AA8EB0607974228BF1746402F1BD950
:105CE00005F1400355F8042B9D4240F8042BF9D1EF
:105CF000A36A40364033A362D4E90A239A4204D30C
:105D0000E16920460439FFF795FF8BF3118846457A
:105D1000D9D28AF31188CDE729463A46FBF7DEFB54
:105D2000A36A3D443E443B44A362E5E7D0E9042333
:105D30009A4217D1C3689BB1836A8BB1043B9B1A0B
:105D40000ED01360C368013BC360C3691A44836902
:105D50009A42026124BF436A0361002383620123E4
:105D6000184670470023FBE700F0F6B8034B00220B
:105D700058631A610222DA60704700BF000C0040CD
:105D8000014B0022DA607047000C0040014B586361
:105D9000704700BF000C0040014B586A704700BFBD
:105DA000000C0040024B034A1A60034A5A607047D5
:105DB000D84D0020684E002000000220074B4942C9
:105DC00010B55C68201A08401968821A914203D8FD
:105DD000944201D35A6010BD0020FCE7D84D00204A
:105DE00008B5202383F31188FFF7E8FF002383F32E
:105DF000118808BD4B6843608B688360CB68C360C3
:105E00000B6943614B6903628B6943620B680360F2
:105E10007047000008B5354B40F2FF70D3F8E01032
:105E20000143C3F8E010D3F8082102433048C3F817
:105E30000821304AD3F808311146FFF7DBFF00F59F
:105E4000806002F11C01FFF7D5FF00F5806002F1D0
:105E50003801FFF7CFFF00F5806002F15401FFF732
:105E6000C9FF00F5806002F17001FFF7C3FF00F584
:105E7000806002F18C01FFF7BDFF00F5806002F148
:105E8000A801FFF7B7FF00F5806002F1C401FFF73A
:105E9000B1FF00F5806002F1E001FFF7ABFF00F514
:105EA000806002F1FC01FFF7A5FF02F58C7100F59F
:105EB0008060FFF79FFF00F00BF90F4BD3F89022A3
:105EC00042F00102C3F89022D3F8942242F001027A
:105ED000C3F894220522C3F898204FF06052C3F80B
:105EE0009C20064AC3F8A02008BD00BF0044025809
:105EF00000000258906B000800ED00E01F0008034E
:105F000008B500F0FDFAFEF72DF8104BD3F8DC20B1
:105F100042F04002C3F8DC20D3F8042122F0400212
:105F2000C3F80421D3F80431094B1A6842F008027F
:105F30001A601A6842F004021A60FEF755FEFEF776
:105F4000BFFCBDE80840FEF75DBA00BF0044025840
:105F50000018024870470000114BD3F8E82042F0C7
:105F60000802C3F8E820D3F8102142F00802C3F871
:105F700010210C4AD3F81031D36B43F00803D363DC
:105F8000C722094B9A624FF0FF32DA6200229A610F
:105F90005A63DA605A6001225A611A60704700BF82
:105FA000004402580010005C000C0040094A08B58B
:105FB0001169D3680B40D9B29B076FEA01011161E7
:105FC00007D5202383F31188FDF7FCFF002383F31B
:105FD000118808BD000C004008B53C4B4FF0FF3164
:105FE000D3F8802062F00042C3F88020D3F88020EC
:105FF00002F00042C3F88020D3F88020D3F8842038
:10600000C3F88410D3F884200022C3F88420D3F886
:106010008400D86F40F0FF4040F4FF0040F43F5050
:1060200040F03F00D867D86F20F0FF4020F4FF0019
:1060300020F43F5020F03F00D867D86FD3F8880095
:106040006FEA40506FEA5050C3F88800D3F88800D8
:10605000C0F30A00C3F88800D3F88800D3F8900092
:10606000C3F89010D3F89000C3F89020D3F89000B4
:10607000D3F89400C3F89410D3F89400C3F8942094
:10608000D3F89400D3F89800C3F89810D3F8980088
:10609000C3F89820D3F89800D3F88C00C3F88C107C
:1060A000D3F88C00C3F88C20D3F88C00D3F89C0074
:1060B000C3F89C10D3F89C10C3F89C20D3F89C30F4
:1060C000FEF7E8FEBDE8084000F0E6B900440258DB
:1060D000614B0122C3F80821604BD3F8F42042F051
:1060E0000202C3F8F420D3F81C2142F00202C3F8E4
:1060F0001C210222D3F81C31594BDA605A689104F2
:10610000FCD5584A1A6001229A60574ADA60002288
:106110001A614FF440429A61514B9A699204FCD53E
:106120001A6842F480721A604C4B1A6F12F4407F66
:1061300004D04FF480321A6700221A671A6842F0BE
:1061400001021A60454B1A685007FCD500221A61FB
:106150001A6912F03802FBD1012119604FF0804119
:1061600059605A67414ADA62414A1A611A6842F430
:1061700080321A60394B1A689103FCD51A6842F4D0
:1061800080521A601A689204FCD53A4A3A499A62D7
:1061900000225A6319633949DA6399635A64384AA9
:1061A0001A64384ADA621A6842F0A8521A602B4B15
:1061B0001A6802F02852B2F1285FF9D148229A6198
:1061C0004FF48862DA6140221A622F4ADA644FF093
:1061D00080521A652D4A5A652D4A9A6532232D4AF6
:1061E0001360136803F00F03022BFAD11B4B1A69DB
:1061F00042F003021A611A6902F03802182AFAD131
:10620000D3F8DC2042F00052C3F8DC20D3F804219C
:1062100042F00052C3F80421D3F80421D3F8DC2063
:1062200042F08042C3F8DC20D3F8042142F08042DF
:10623000C3F80421D3F80421D3F8DC2042F0004253
:10624000C3F8DC20D3F8042142F00042C3F8042153
:10625000D3F80431704700BF008000510044025859
:106260000048025800C000F0020000010000FF01D9
:1062700000889008225050003F02090147020400A4
:106280002F040407BD0BFF01200000200010E000D8
:1062900000010100002000524FF0B04208B5D2F8D2
:1062A000883003F00103C2F8883023B1044A136830
:1062B0000BB150689847BDE80840FEF7E3BC00BF4B
:1062C000E04D00204FF0B04208B5D2F8883003F01E
:1062D0000203C2F8883023B1044A93680BB1D06836
:1062E0009847BDE80840FEF7CDBC00BFE04D002058
:1062F0004FF0B04208B5D2F8883003F00403C2F87A
:10630000883023B1044A13690BB150699847BDE83E
:106310000840FEF7B7BC00BFE04D00204FF0B04290
:1063200008B5D2F8883003F00803C2F8883023B1EA
:10633000044A93690BB1D0699847BDE80840FEF75D
:10634000A1BC00BFE04D00204FF0B04208B5D2F82C
:10635000883003F01003C2F8883023B1044A136A6E
:106360000BB1506A9847BDE80840FEF78BBC00BFF0
:10637000E04D00204FF0B04310B5D3F8884004F44E
:106380007872C3F88820A30604D5124A936A0BB129
:10639000D06A9847600604D50E4A136B0BB1506B58
:1063A0009847210604D50B4A936B0BB1D06B9847E5
:1063B000E20504D5074A136C0BB1506C9847A3054E
:1063C00004D5044A936C0BB1D06C9847BDE81040DB
:1063D000FEF758BCE04D00204FF0B04310B5D3F8A5
:1063E000884004F47C42C3F88820620504D5164A2C
:1063F000136D0BB1506D9847230504D5124A936D68
:106400000BB1D06D9847E00404D50F4A136E0BB161
:10641000506E9847A10404D50B4A936E0BB1D06E11
:106420009847620404D5084A136F0BB1506F984720
:10643000230404D5044A936F0BB1D06F9847BDE88D
:106440001040FEF71FBC00BFE04D002008B5034818
:10645000FCF7C8FBBDE80840FEF714BC0825002087
:1064600008B50348FCF7ACFCBDE80840FEF70ABCE1
:106470002825002008B50348FCF7A2FCBDE8084029
:10648000FEF700BC9425002008B5FFF78FFDBDE89E
:106490000840FEF7F7BB0000062108B50846FFF7E5
:1064A00083FA06210720FFF77FFA06210820FFF76D
:1064B0007BFA06210920FFF777FA06210A20FFF769
:1064C00073FA06211720FFF76FFA06212820FFF73D
:1064D0006BFA09217A20FFF767FA0A215C20FFF79F
:1064E00063FA07213220FFF75FFA0C212520FFF71E
:1064F0005BFA0C215220BDE80840FFF755BA0000B6
:1065000008B5FFF769FD00F00FF8FCF76BFEFDF72B
:1065100043F8FCF715FFFDF7D5FAFFF71BFDBDE8C3
:106520000840FFF721BC00000023054A194601334B
:10653000102BC2E9001102F10802F8D1704700BF28
:10654000E04D00200B460146184600F027B8000039
:10655000FEF7EEB9FFF7FCBF012838BF012010B5E8
:1065600004462046FEF7A4F930B900F007F808B950
:1065700000F00CF88047F4E710BD0000024B1868EB
:10658000BFF35B8F704700BF604E002008B5062048
:1065900000F04AF80120FDF783FE000010B5054C1D
:1065A00013462CB10A4601460220AFF3008010BD0D
:1065B0002046FCE70000000010B50139024490427B
:1065C00001D1002005E0037811F8014FA34201D06A
:1065D000181B10BD0130F2E71F2938B504460D46DF
:1065E00004D9162303604FF0FF3038BD426C12B15E
:1065F00052F821304BB9204600F030F82A460146C7
:106600002046BDE8384000F017B8012B0AD0591CCD
:1066100003D1162303600120E7E7002442F8254058
:10662000284698470020E0E7024B01461868FFF72C
:10663000D3BF00BF6822002038B5074D00230446B1
:10664000084611462B60FDF72FFE431C02D12B6834
:1066500003B1236038BD00BF644E0020FDF71EBEAD
:10666000034611F8012B03F8012B002AF9D17047DA
:106670000000000001000000000100010000000017
:1066800000000000000000005265717565737465BC
:106690006420746F206572617365206D6F72652070
:1066A0007468616E2077652063616E0A00457261CF
:1066B000736520436F6D6D616E642052656365691B
:1066C0007665640A0050435420444F4E453A2025D5
:1066D000640A000053544D333248373F3F3F005364
:1066E000544D3332483734332F37353300000000F0
:1066F00001105A00031059000120580003205600D1
:10670000773235710000000000000000000000003A
:10671000000000000000000045170008751A00087E
:10672000751A0008491700084D170008511700088E
:1067300055170008751A0008751A0008751A000820
:106740006D170008711700088917000891170008D5
:106750009D170008A1170008A517000808250020AC
:10676000010000000000000000000000C518000843
:10677000DD18000845170008B117000811190008B6
:10678000CD170008A9190008D919000855170008E5
:10679000C9170008B5170008C51700086D170008CD
:1067A0007117000889170008911700089D17000845
:1067B000A1170008A5170008000000000000000055
:1067C00045180008A9170008AD17000853464450A3
:1067D000000000004A454445433A204661696C6523
:1067E0006420746F2064657465637420666C6173E3
:1067F00068206465766963653A2025730A004A4516
:106800004445433A204661696C656420746F206397
:106810006F6E66696720666C61736820646576696F
:1068200063653A2025730A004A454445433A2044AB
:106830006574656374656420466C617368204465A3
:10684000766963653A2025730A0045787420466CA2
:10685000617368204E6F7420466F756E642100006E
:106860006D7432357100773235712D6474720000A9
:106870006068000820BA000000670008EF400000D0
:1068800066680008EF7000000000000000000000D3
:1068900055210008B5230008911A0008951A000830
:1068A0003D1B00081D230008991A00089D1A0008C6
:1068B000152200080D1B000875220008791F00082A
:1068C000A51A0008A11A000845240008051B0008A5
:1068D0000000000000000000092500081125000844
:1068E000F5240008FD2400082125000825250008BE
:1068F000286E756C6C29000000000000B9290008A2
:106900009129000859290008752900084D444D4176
:10691000206661696C7572650000000000960000D9
:106920000000000000000000000000000000000067
:106930000000000000000000AD310008993100089F
:10694000D5310008C1310008CD310008B931000847
:10695000A531000891310008E13100080000000075
:10696000BD320008A9320008E5320008D132000823
:10697000DD320008C9320008B5320008A132000833
:10698000F1320008000000000100000000000000DB
:106990006D61696E0000000069646C6500000000B4
:1069A00098690008582E0020D02F00200100000018
:1069B000613F0008000000004172647550696C6F0F
:1069C000740025424F415244252D424C0025534529
:1069D0005249414C25000000020000000000000068
:1069E000DD3400084D3500084000400078480020A4
:1069F00088480020020000000000000003000000A2
:106A000000000000953500080000000010000000A4
:106A10009848002000000000010000000000000075
:106A2000884C002001010200A1430008B142000887
:106A30004D4300083143000843000000406A00084D
:106A400009024300020100C03209040000010202F1
:106A500001000524001001052401000104240202A4
:106A60000524060001070582030800FF0904010050
:106A7000020A00000007050102400000070581022C
:106A800040000000120000008C6A00081201100192
:106A900002000040091241570002010203010000F8
:106AA0000403090425424F415244250044657645BC
:106AB000426F7848377632003031323334353637EA
:106AC00038394142434445460000000000000020A0
:106AD000000002000200000000000030000004007E
:106AE0000000000000000024000008000400000076
:106AF0000004000000FC0000020000000000043060
:106B000000800000000000000000003800000100CC
:106B1000010000004000005280000052C0000052FE
:106B2000000100524001005280010052C001005299
:106B3000000200524002005280020052C002005285
:106B4000000300524003005280030052C003005271
:106B50000004005200000000E9360008A1390008D6
:106B60004D3A000840004000C04D0020C04D0020BC
:106B700001000000D04D0020800000004001000016
:106B800008000000000100000004000008000000F0
:106B90000401A82A00000000AAAAAAAA000114243D
:106BA000FDFF00000000000070A70A002020000088
:106BB00000000000AAAAAAAA00000000FFFF00002F
:106BC0000009000A000000000000000000000000B2
:106BD000AAAAAAAA00000000FFFF0000000000000F
:106BE000000000000000800A00000000AAAAAAAA73
:106BF00000000000FFFF000000000000009099006E
:106C00002080020000000000AAAAAAAA00400100F9
:106C1000FFFF0000000900700700000000000000F6
:106C200000000000AAAAAAAA00000000FFFF0000BE
:106C30000000000000000000000000000000000054
:106C4000AAAAAAAA00000000FFFF0000000000009E
:106C5000000000000000000000000000AAAAAAAA8C
:106C600000000000FFFF0000000000000000000026
:106C70000000000000000000AAAAAAAA000000006C
:106C8000FFFF000000000000000000000000000006
:106C900000000000AAAAAAAA00000000FFFF00004E
:106CA00000000000000000000000000000000000E4
:106CB000AAAAAAAA00000000FFFF0000000000002E
:106CC000000000001C96FF7F010000000000000093
:106CD0002504000000000000000000000000690022
:106CE000FF000000D02F0020282500209425002040
:106CF00000000000D46600083F00000050040000BF
:106D0000DF6600083F000000009600000000080059
:106D1000960000000008000004000000A06A0008BF
:106D20000000000000000000000000000000000063
:106D300000000000000000006C22002000000000A5
:106D40000000000000000000000000000000000043
:106D50000000000000000000000000000000000033
:106D60000000000000000000000000000000000023
:106D70000000000000000000000000000000000013
:106D80000000000000000000000000000000000003
:0C6D9000000000000000000000000000F7
:00000001FF
